:020000040800F2
:100000006842002031940008B5900008B7900008BD
:10001000B9900008BB900008BD90000800000000E7
:10002000000000000000000000000000398000080F
:10003000BF90000800000000E17F0008657F000815
:10004000699400086D940008719400087594000884
:10005000799400087D940008819400088594000834
:10006000899400088D94000891940008C1900008BC
:1000700095940008999400089D940008A1940008A4
:10008000A5940008A9940008AD940008B194000854
:10009000B5940008B9940008BD940008C194000804
:1000A000C5940008C7900008C9940008CD940008C2
:1000B000D1940008D5940008D9940008DD94000874
:1000C000E1940008E5940008E9940008ED94000824
:1000D000F1940008D9900008F594000815910008E3
:1000E000F9940008FD9400080195000805950008A2
:1000F000099500080D950008119500081595000850
:10010000199500081D9500082195000825950008FF
:10011000299500082D9500083195000835950008AF
:10012000399500083D95000841950008459500085F
:10013000499500084D95000851950008559500080F
:10014000599500085D9500086195000865950008BF
:10015000699500086D950008539100087195000895
:1001600075950008799500087D950008819500082F
:1001700085950008899500088D950008000000000D
:100180009195000895950008999500089D9500089F
:10019000A1950008A5950008A9950008AD9500084F
:1001A000B1950008B5950008B995000840F0200009
:1001B00070472DE9F14FB0B0924604910DF1420124
:1001C0003A9A2B9199464A7000200AE01AF8011BCE
:1001D0000498309A90470028049000F034860D98D7
:1001E000401C0D909AF8000050B12528EED1002156
:1001F00000220791089209910A920B910C9204E057
:100200000D9800F022BE41F001011AF8010F2028DC
:10021000F9D023280CD02B2804D02D2805D0302845
:1002200009D00BE041F00201EFE741F00401ECE7F7
:1002300041F00801E9E741F01001E6E72A280FD173
:10024000D9F8002052F8040BC9F8002000280F90BC
:1002500003D540420F9041F004010AF1010A14E075
:100260000F92DFF8EC3B0AE00F98984205DA00EBBA
:10027000800402EB4402303A0F920AF1010A9AF824
:100280000020A2F130000A28EED39AF800002E28B0
:1002900003D04FF0FF320E9229E01AF8010F2A28FE
:1002A00009D1D9F8000050F8042BC9F800000E92CB
:1002B0000AF1010A1BE02D280CBF0AF1010A0020F7
:1002C00000220E92DFF8884B0BE040B90E9AA24252
:1002D00005DA02EB820503EB4503303B0E930AF18E
:1002E000010A9AF80030A3F130020A2AEDD3ADF8E2
:1002F00040100FF660309AF8001000F0EDFE08B1E3
:100300001AF8010B8DF842009DF84200682805D1CB
:100310009AF8000068280CD1622106E06C2804BF1E
:100320009AF800006C2804D171218DF842100AF16E
:10033000010A12A806901AF801BBBBF125012CD0C6
:100340001C3900F09481091F022940F29081133971
:1003500000F0AB84093900F08A81891E00F04085E5
:10036000491E00F0ED84491E022940F28081091FD8
:1003700000F0E684491F00F0EF80491E00F09584EC
:10038000491E00F0D780C91E0CD0891E00F08D8454
:10039000C91E00F08A8400F02EBD01230793252199
:1003A00000F026BDD9F8000050F8044BC9F8000051
:1003B000002C059440F0AB802B994878002800F081
:1003C000A1804FF0FF340FF6942000F095FE241A20
:1003D00040F0398500F01BBD01236A4602A9304672
:1003E00000F000FE002840F02E85641EF4D1309607
:1003F000079C12AF74B1309E17F8011B0498B047E8
:100400000028049000F01F850D98401C641E0D907C
:10041000F2D130960A9C3021002C8DF800100CDDB2
:10042000309E01236A4602A9304600F0DBFD002819
:1004300040F00985641EF4D13096059F089C74B184
:10044000309E17F8011B0498B0470028049000F074
:10045000FA840D98401C641E0D90F2D130960B9CCE
:100460003021002C8DF800100CDD309E01236A46EF
:1004700002A9304600F0B6FD002840F0E484641E76
:10048000F4D1309605980899099C471874B1309EAC
:1004900017F8011B0498B0470028049000F0D3849B
:1004A0000D98401C641E0D90F2D130960C9C3021AA
:1004B000002C8DF800100CDD309E01236A4602A945
:1004C000304600F08FFD002840F0BD84641EF4D15A
:1004D00030969DF8400041077FF584AE2020002D26
:1004E0008DF800007FF77EAE309C01236A4602A99A
:1004F000204600F077FD002840F0A5846D1EF4D161
:1005000030946FE60FF63C30059000F080BC0E9DF5
:10051000002D04D5204600F00FFE044607E02A46D1
:10052000204600F013FE002814BF041B2C4608943C
:1005300000F06DBCD9F8001051F8040BC9F8001098
:1005400020F00004002121F0FF35CDE9024512AB77
:100550000593782100F040BC2B99487820B14FF0EA
:10056000FF340FF6B02030E79DF84200622860D0DB
:10057000682817D06A283FD06C2806D0712847D049
:1005800074282CD07A281DD062E0D9F8001051F8D8
:10059000040BC9F80010002866D14FF0FF340FF6A5
:1005A0008C2012E7D9F8001051F8040BC9F800109C
:1005B00020B94FF0FF340FF6742006E70D99018043
:1005C00000F025BCD9F8001051F8040BC9F8001050
:1005D000002849D14FF0FF340FF65020F5E6D9F846
:1005E000001051F8040BC9F8001000283CD14FF05E
:1005F000FF340FF63820E8E6D9F8001051F8040B64
:10060000C9F8001080B94FF0FF340FF62020DCE667
:10061000D9F8001051F8040BC9F8001020B94FF0B8
:10062000FF340FF60820D0E60D9AD317C0E9002357
:10063000EDE3D9F8001051F8040BC9F8001020B907
:100640004FF0FF340FF6E410BFE60D990170DEE3C2
:10065000D9F8001051F8040BC9F8001020B94FF078
:10066000FF340FF6C810B0E60D990160CFE39DF896
:1006700042004C2807BFD9F80010CA1DD9F8000065
:10068000C21D22F00702C9F80020D2E90001083299
:10069000C9F80020CDE90201C80F02D007982D212A
:1006A0000AE0BDF84000810702D507982B2103E03E
:1006B000C00705D50798202112AA1154401C0790A5
:1006C00012A807994BF0200300EB010CDDE90201B1
:1006D000CDE92C01612BCDF814C021AC0BD00E98C4
:1006E000002848BF062105D404BF4BF0200067282E
:1006F00001D101210E91DDE902014F0047EAD077D7
:100700007E15FF174FF0FF32974208BF964210D177
:10071000090341EA10510003002908BF002808D04E
:10072000ABF1610503211A2D089118D30FF61C11A6
:1007300010E0DDE902014A00521512F1010F11D15A
:1007400008030FD1ABF1610503211A2D08911FD3C6
:100750000FF600110322604600F024FD57E30FF668
:10076000E801F7E7DDE902016A4600F027FDCDE97F
:1007700002014BF02000612811D105983021017051
:10078000821C0592BBF1610F0CBF7821582102E059
:100790000FF6BC01DEE741700798801C0790DDE989
:1007A000020120F0000231F0004308BF002A02D10C
:1007B0000026002542E14BF02008B8F1610F40F01F
:1007C00092800E98002847BF21210191401C019082
:1007D000019FDDE92C017F1C00220023DDE9024599
:1007E00000F024FD38BF85F0004500998DF8842085
:1007F000091F002F00910DF1850632DD20462946A4
:100800000022002300F02CFD2BD21C2200F042FD20
:1008100004460D4600F0DCFDFF1F002F804609DD79
:1008200000F0F2FD02460B462046294600F0BCFED1
:1008300004460D46F01D0721B8F1000F0CDD491EDE
:100840005EBF08F00F0200F8012D4FEA2818F3D51B
:1008500002E0002200F8012D491EFAD5C61D002F26
:10086000CCDC0DF18500361A01980DF18504864225
:10087000D8BF304600282FD4B04206DA0DF18501EA
:100880000A5C082AA8BF0F2100DA0021024621AB2A
:10089000134400E0401E13F80159521E8D42F9D056
:1008A0000F2904D10DF185018B5C5B1C8B54002A50
:1008B00004D50099091D21AC401C0091411E0BD4A8
:1008C000621813783033DDB23A2DA4BF5B443A3B53
:1008D000491E02F80139F4D50E99002940F1AC8087
:1008E000421E0E92A8E00099DFF8E82647F29750E2
:1008F000414391FBF2F20092DDE92C45C2F107027F
:10090000002A25F0004504DD2046294600F03EFB84
:100910000BE052420020DFF8C01600F037FB024621
:100920000B462046294600F0B1FE04460D46B8F1BC
:10093000660F06BF009F0A3706270E983F18142F30
:10094000C8BF142730208DF884000DF18506002FD4
:1009500034DD2046294600F0BDFF01460A4606F177
:10096000080304200A26B2FBF6F606EB860EA2EB7D
:100970004E02303203F8012C0A22B6FBF2F202EBEF
:10098000820EA6EB4E063036401E03F8026DE9D10A
:10099000083F002F03F10806D9DD084600F0ACFF40
:1009A00002460B462046294600F0FEFD0022DFF8F5
:1009B0002C3600F0AFFF04460D46CAE70DF1850066
:1009C000361A0DF1850404E00098401E761E009052
:1009D000641C20783028F7D0B8F1660F02D1009857
:1009E000401C04E0B8F1650F0CBF012000200E99F7
:1009F00040188642B8BF701E00281DD4B04204DAE9
:100A0000215C3429C8BF392100DC30210246631E35
:100A10009D1800E0401E15F80169521E8E42F9D063
:100A2000392902D1A15C491CA154002A04D500999E
:100A3000491C1C46401C00910646009D0E9F30B28A
:100A4000002802DC01260FF210644BF0200066281B
:100A500008BF6D1C15D067280FFA85F841D118F131
:100A6000040F44DBB84542DA9DF840006D1C0107D5
:100A700003D430B2B842D8BF074628B23F1A48BFA5
:100A800000270FFA85F8B8F1000F00F3AF8008983F
:100A9000411C0891302205990A54002F03DC9DF86F
:100AA0004000010705D50898411C08912E220599A0
:100AB0000A5417EB080FB8BF7D422DB26842ED19FA
:100AC00032B20B909542B8BF2E46059B089836B2BD
:100AD000099632462146184400F064FBAD1B0C9584
:100AE000CCE0BBF1610F15D14FF0700B17E030B2C5
:100AF000B84204DA9DF840100A0758BF07467F1E27
:100B000048BF0027BBF1670F14BF4FF0450B4FF0F4
:100B1000650B04E0BBF1410F08BF4FF0500B089884
:100B2000411C0891002F059914F8012B0A5403DC8D
:100B30009DF84000010719D50898411C08912E2204
:100B400005990A54002F11DD761E30B28742B8BFD6
:100B50003E460598089B32B22146184400F022FB1D
:100B6000089836B23018BF1B08900B970598089963
:100B70000844B8F1000F80F800B003D42B22427073
:100B8000821C04E02D2145464170821C6D420021EB
:100B90002CAB28460AE004460A2094FBF0F000EB58
:100BA0008005A4EB450403F8014B491C00B2002862
:100BB000F1DC012906DC4BF02000652804BF302061
:100BC00002F8010B00292CAB08D1302002F8010BF0
:100BD00006E0491E585C303002F8010B0029F8DCB1
:100BE000059908980844121A099247E030B229B2D0
:100BF00088421BDA0598089B32B22146184400F05F
:100C0000D1FA089936B271180891A8EB0600002FA6
:100C10000B9003DC9DF84000020705D5059A2E20B5
:100C200050540999491C09910C9727E00598089B95
:100C30002AB22146184400F0B5FA0898761B4044C1
:100C4000002F089003DC9DF840100A0704D5411CD2
:100C500008912E2205990A5430B28742B8BF3E4609
:100C60000598089B32B204EB0801184400F09AFA88
:100C7000089836B23018BE1B08900B969DF84000BD
:100C800000F01400102840F0C280079A08980B99D1
:100C9000821809988A1882180C980F99801888422F
:100CA00080F2B580081A0A90B1E09DF842006228EF
:100CB00008D068280ED06A2814D06C281FD071285C
:100CC00010D01CE0D9F8001051F8040BC9F800103E
:100CD000C0B21AE0D9F8001051F8040BC9F800109E
:100CE00080B212E0D9F80000C21D22F00702C9F854
:100CF0000020D2E900010832C9F8002006E0D9F846
:100D0000001051F8040BC9F800100021CDE90201D0
:100D10009DF8400001075AD5DDE90223002B08BFEA
:100D2000002A54D04BF02000782850D1079812A9FF
:100D300030220A54401C431C079301F800B046E0DF
:100D40009DF84200622808D068280ED06A2814D086
:100D50006C281FD0712810D01CE0D9F8001051F871
:100D6000040BC9F8001040B21AE0D9F8001051F88D
:100D7000040BC9F8001000B212E0D9F80000C21D3F
:100D800022F00702C9F80020D2E900010832C9F8B0
:100D9000002006E0D9F8001051F8040BC9F8001043
:100DA000C117CDE90201002902D507982D210AE0DB
:100DB000BDF84000810702D507982B2103E0C0074A
:100DC00005D50798202112AA1154401C079012A89B
:100DD000079901440591594602A800F04DF816E024
:100DE00001200790D9F8000050F8041BC9F8000052
:100DF0008DF848100BE001212522BBF1000F07916F
:100E00008DF8482003D0022207928DF849B00F9D3B
:100E100007990A986D1A08992D1A0B986D1A099955
:100E20002D1A0C986D1A9DF840102D1A48073FF5A1
:100E3000DFAA2021002D8DF800107FF7D9AA309E5F
:100E40002C46FFF7C9BA4FF0FF3031B0BDE8F08F44
:100E5000CBCCCC0C686A6C747A4C00007072696EF2
:100E600074665F733A206261642025732061726743
:100E7000756D656E740000002DE9FC4707468A46D3
:100E80003C6950466F2808BF082505D0FFF78EF94A
:100E9000782814BF0A251025D7E900013C26804692
:100EA0008946BAF1640F18BFBAF1690F05D100295C
:100EB00003D5D8F1000869EB4909B9F1000F08BF63
:100EC000B8F1000F0CD1386B50B9082D3AD197F812
:100ED0003800010736D530223B2684F83B2031E02C
:100EE0008DF800A0404649462A46EB1700F0E8FD81
:100EF0003032D0B2761E3A2801960EDAA25540461C
:100F000049462A46EB1700F0DBFD80465FEA0109FF
:100F100008BFB8F1000F05D108E09DF800001218D5
:100F2000513AEBE7F868A1198842DBD3082D09D1C3
:100F300097F83800010705D5A05D302802D0761E4D
:100F40003020A055C6F13C03BB61A119F960386B94
:100F5000834208DAC31A3B624FF6EF70398F0140C3
:100F60003987BDE8F38700280ED597F8380000F0E0
:100F70001400102808D17A6B7969386A521A121A4B
:100F8000D21A002AC8BF3A62BDE8F3872DE9D043E0
:100F900006460F4614464FF00008DFF8449012E072
:100FA000E00707D542464B463046394600F0B2FCD2
:100FB00006460F464046494642464B4600F0AAFCCC
:100FC000641080468946002CEAD130463946BDE897
:100FD000D0830000A08601000000F03F84D7974135
:100FE00000002440F8B505460E4617461C46002072
:100FF0005CB117F8011BB068A847B06030B1F06A67
:10100000401CF0620020641EF3D1F2BD4FF0FF30AF
:10101000F2BD00007072696E74665F733A20256ECF
:1010200020646973616C6C6F776564007072696EBF
:1010300074663A2062616420256E20617267756D66
:10104000656E7400000000006E616E004E414E003F
:10105000696E6600494E46003000F0B402461068E2
:1010600095681318506803EB5004C00748BF4D44FF
:10107000A3422DD013F8016B16F0030004BF13F840
:10108000010BC01C31090F2907D113F8011B0F31C7
:1010900003E013F8017B05F8017B401EF9D100291C
:1010A000E6D013F8010BC6F38106032E08BF13F830
:1010B000016B00EB0620404228440026B71E8F42F9
:1010C0001EBF10F8017B05F8017B761CF6D1CFE737
:1010D000F0BC02F10C007047C9B202788A421AB122
:1010E0001CBF10F8012FF9E718BF002070470268F5
:1010F000531C03601170704780B500B906A0054904
:101100000B681BB122220021984701E000F05BFD33
:10111000222002BD603E0020636F6E7374726169AD
:101120006E742068616E646C65723A20626164203E
:101130006D6573736167650000F1010310F8011BB1
:1011400011B110F8011BFBE7C01A7047C9B2830741
:1011500006D0521E22D310F8013B9942F7D11FE06E
:10116000083A13D302F1040241EA012141EA0141A4
:1011700050F8043B121F21BF4B40A3F1013C2CEA65
:10118000030C1CF0803FF3D0C9B2001F083210F8E6
:10119000013B521E28BF91EA030FF8D818BF012067
:1011A000401E70474AB1000011F8013B521E00F882
:1011B000013B1CBF11F8013BF8E7704710B514461E
:1011C00000F002F8226010BDC1F30A5343B14A0097
:1011D00012F5001F28D2A3F2FE32A1EB0251704794
:1011E00050EA410C20D001F0004C31EA0C01B1FA78
:1011F00081F204BFB0FA80F3D2180B3AB2F12003A7
:101200002CBF00FA03F1914041EA0C013EBFC2F14C
:10121000200C20FA0CF319439040524240F2FD3367
:10122000D21A01EB035170470022704741EA030CC8
:1012300050EA4C0C52EA0C0C4FF4001C09D307D0B6
:101240001CEB410F9CBF1CEB430F8B4208BF82423B
:1012500070471CEB430FFBD8994208BF9042704780
:1012600041EA030C50EA4C0C52EA0C0C4FF4001CFF
:1012700009D307D01CEB410F9CBF1CEB430F9942D5
:1012800008BF904270471CEB410FFBD88B4208BF50
:1012900082427047124254D440F2FF7C1CEA115340
:1012A0000FD0634531D09B1863453CBF01EB025121
:1012B000704701F0004141EA0C510020AFF300807B
:1012C000704750EA410320D001F0004C91EA0C0134
:1012D0001CD0B1FA81F30B3B9A420DD9D21A994036
:1012E00051EA0C01C3F1200C20FA0CFC6144984037
:1012F000531C40F2FF7CD7E7914041EA0C01C2F158
:10130000200C20FA0CF3194390407047B0FA80F398
:101310001533202BE0D3202AEED3203A203B9A42EB
:1013200009D9D21A00FA03F141EA0C010020531C3A
:1013300040F2FF7CB8E700FA02F141EA0C0100201C
:101340007047524240F2FF7C1CEA11530DD06345B6
:10135000DBD0B2EB030C3CBFA1EB025170470CF1A8
:10136000010221EA035141F4801150EA410CCCD032
:1013700001F0004C352A27DC30B481EA0C01B2F1CF
:10138000200309DAC2F12003044601FA03F5D04034
:101390002843D1409C400CE0C3F12002450020FAD4
:1013A00003F418BF44F0010421FA03F091400C4308
:1013B000002174F1004550F1000051EB0C01244272
:1013C00030BC7FF47BAF70476146002076E70000B9
:1013D000C1F30A5340F21E42D31A0CDDCA0283F352
:1013E000070342EA505242F00042DA4002EBE17257
:1013F00082EAE17070476FEAE17203F2E13008B10E
:1014000082F000407047000010F0004160B148BF1A
:101410004042B0FA80F29040D21CC2F5846241EAA8
:10142000025202EBD02140057047000070B491EAEF
:10143000030F4FF0004540F1BF806B40841A71EB01
:10144000030604D26E40001BB141121973414FF4E0
:10145000001C1CEB410F34BF7CEB430683E00C0DFA
:10146000A4EB1356362E00F37C80012E45EAC323ED
:1014700041DC43EA525312BFD20292025B082405B8
:1014800045EAC12141EA5051D2EBC020994125D40F
:1014900007D1B0FA80F610FA06F162D000202036AB
:1014A00008E0B1FA81F6B140C6F1200220FA02F25A
:1014B0001143B0404FEAF474B4EB465434F00106E3
:1014C0004FEA74040AD8D6F50016760D04F00044ED
:1014D000F04061FA06F25040F1404840C00A40EA4C
:1014E000415021F0004128BF5FEA500550F1000053
:1014F00044EBD12135E0DB0A45EAC121C90AB6F146
:1015000020050EDD42EA0242120CC5F1200603FA64
:1015100006F6EB4042EA06056D42984161F1000192
:101520000DE062FA06F5F240554063FA06FC82EAE5
:101530000C02F3405A406D42904161EB030111F4FB
:10154000801F05D1641E620502D06D0040414941F3
:1015500021F48011430875F1004350F1000041EB84
:10156000045170BC70471CEB410F15D223F00043AF
:1015700052EA43060BD04FEA4C0CBCEB410F04D8A7
:101580000C0D661E342EB7DDEBE7801A994150EA48
:10159000410608BF0021E4E708BF1CEB430F28BF4A
:1015A0006FF00001DDE7000070B491EA030F4FF027
:1015B00000457FF543AF6B40841A71EB030603D2FD
:1015C000001BB141121973414FF4001C1CEB410F79
:1015D00034BF7CEB430442E00C0DA4EB1356352ED4
:1015E0004FDC45EAC323DB0A45EAC121C912B6F143
:1015F00020050DDD63FA05F6EB4086EA030512428D
:1016000018BF45F00105C01851F100010CD213E0DC
:1016100062FA06F5F2405540F3415A40B340F340B8
:101620005A408018594107D349085FEA30005FEA01
:10163000350528BF45F0010501F58011420875F117
:10164000004250F1000041EB04514E0016F5001F1E
:1016500070BC38BF70470020090D090570471CEBAE
:10166000410F10D252EA43060BD0BCEB410F05D814
:101670000C0DAB43661E342EB6DD02E0AB43801882
:10168000594170BC704770BC70470000F0B540F223
:10169000FF7581EA030C0CF0004C15EA11541DBFD4
:1016A00015EA1357AC42AF42E5E0BC41C1F3130168
:1016B000C3F31303801A994143F4801304D2641EC8
:1016C0000018494180185941C90241EA5051B1FB03
:1016D000F3F603FB1611A2FB0675D7EBC020A94158
:1016E00002D2761E80185941C90241EA5051B1FB1D
:1016F000F3FE03FB1E11A2FB0E75D7EBC020A94120
:1017000003D2AEF1010E80185941890241EA90518D
:10171000760546EA8E2EB1FBF3F603FB1611A2FB0B
:101720000675D7EB8020A94102D2761E8018594158
:10173000C90241EA50514EEA060EB1FBF3F603FB33
:101740001611A2FB0675D7EBC020A94102D2761E66
:1017500080185941C90241EA5051B1FBF3F703FB2C
:101760001711A2FB0735D3EBC020A94167F1000791
:101770000CBF004247F0010766F3D5274FEA1E3140
:10178000B80814F5806412DDBD0775F1004250EB16
:101790000E5051EB045111F5801F5CBF41EA0C0162
:1017A000F0BD4CF07F6141F0E0410020F0BDBD078D
:1017B0006D0840EA0E5041F48011D4F10104B4F1F7
:1017C00020060ADAC4F120060200E04001FA06F31E
:1017D000E1401843B24015430EE0342C13DCC6F14F
:1017E000200445EA40056D0820FA06F2154321FA67
:1017F00006F0A1400D43002175F1004250F10000B8
:1018000051EB0C01F0BD00205FEA0C01F0BDCFB937
:1018100092185B41B3FA83F704BFB2FA82F6BF199C
:101820000B3FB7F120062FBF02FA06F3BB40C7F10A
:10183000200622FA06F638BF3343BA401CB1E41939
:10184000641E33E77F4231F00041B1FA81F404BFF6
:10185000B0FA80F6A4190B3CB4F120062FBF00FAB1
:1018600006F1A140C4F1200620FA06F638BF314344
:10187000A0403C1B1AE7AC421ABF05EA1357AF421F
:1018800012E050EA41061CBF52EA4306BFE750EAA5
:101890004107304661461CBF41EA0551F0BD52EA9E
:1018A000430C08BFC143F0BD00204FF4001616EBF7
:1018B000410F98BF16EB430F08BF16EB410F24BF33
:1018C000C14305E016EB430F0CBF61464CEA0551DE
:1018D000F0BD0000400D40F21E4C40EAC120BCEBC0
:1018E000115C40F0004003D48CF30701C8407047FE
:1018F0006FEAE1707047000050B1B0FA80F18840A3
:10190000C91CC1F58461090501EBD0214005704770
:101910000146704730B540F2FF7C1CEA11541DBFF0
:101920001CEA1355644565453FE0641981EA030CE0
:101930006FF35F530CF0004C43F48013C90241F085
:10194000004141EA505EC5021100A5FB02020028D9
:101950004FF00000EEFB01204FF00001E3FB0521FA
:1019600018BF42F00102401800214941E3FB0E017B
:10197000A4F580640D0302D292184041494154F10C
:10198000010470DD450872F1004250F1000051EB96
:101990000451A1F5801102D441EA0C0130BD40F29E
:1019A000FF7E4CEA0E51002030BD0CEA1355644511
:1019B00018BF654581EA030C0CF0004C41D050EA99
:1019C000410E1CBF52EA430E02E06146002030BDCA
:1019D00024422C441BD15FEA050EF6D0090302BF56
:1019E00001460020AEF1140EB1FA81F5AEEB05040C
:1019F00001FA05FE0C35C5F1200100FA05F5C840D5
:101A00004EEA000E6FF35F5343F480139CE733F00C
:101A10000043B3FA83F504BFB2FA82FE75440B3D6E
:101A2000641BB5F1200E2FBF02FA0EF3AB40C5F1D7
:101A3000200E22FA0EFE38BF43EA0E03AA40641CB1
:101A40007CE750EA410E14BF52EA430E6FF00001EA
:101A50004FF4001515EB430F8EBF194615EB410FE0
:101A60009DE7B4D830BDD4F10104B4F120050FDAFC
:101A7000C4F12005520828BF42F0010210FA05FE09
:101A800001FA05F57244E2BFE0402843E1400FE06F
:101A9000352C9ADCC5F1200452EA400220FA05F206
:101AA00018BF42F0010231FA05F0A1400A430021BB
:101AB00072F1004250F1000051EB0C0130BD00000A
:101AC000D3BBD9B1B2F5803F5BD2022A1ED98C4676
:101AD000B1FBF2F102FB11C31B0443EA1043B3FB59
:101AE000F2FC02FB1C3380B240EA0343B3FBF2F08A
:101AF00002FB103240EA0C4000237047022A05D94D
:101B00008446B0FBF2F002FB10C270474AB105D127
:101B100000F0010249085FEA30007047002200230C
:101B2000704700F053B80B000200002100207047FE
:101B3000F7D3002200237047904271EB030CF2D3DD
:101B400070B5B1FA81F4B3FA83F52C1BA340C4F14C
:101B5000200532FA05F63343A2405FF00046E64026
:101B600002E05B085FEA3202841A71EB030524BFCE
:101B7000204629467641F4D302000B0030000021B4
:101B800070BD70B5B1FA81F4B2FA82F5C4F12004E7
:101B90006419B4F12006DAD3B2405FF00044F44097
:101BA000002502E052085FEA3303C61A71EB020E09
:101BB00024BF3046714664416D41F3D302000B00EF
:101BC0002000290070BD012000F002B8704700001D
:101BD00080B5AFF30080024A11001820ABBEFBE7CE
:101BE0002600020038B5040001D1012032BD00F00A
:101BF0004DF918B900F085FB00F0D9FE85E090F8AA
:101C00003D10012901D001207047022180F83D10CC
:101C1000DFF82C220168914218BFB1F1804F12D039
:101C2000DFF8202291421CBFDFF81C3299420AD013
:101C3000DFF8182291421FBFDFF814329942DFF813
:101C40001422914209D18B68DFF818121940062935
:101C500018BFB1F5803F05D001680A68084642F018
:101C6000010202600020704701680A6A41F2111304
:101C70001A4202BF096A40F24442114239E090F828
:101C80003D10012901D001207047022180F83D104C
:101C90000168CA6842F00102CA600168DFF8A02149
:101CA000914218BFB1F1804F12D0DFF898219142D4
:101CB0001CBFDFF8943199420AD0DFF8902191429D
:101CC0001FBFDFF88C319942DFF88821914209D19A
:101CD0008B68DFF890111940062918BFB1F5803FD5
:101CE00005D001680A68084642F00102026000203F
:101CF000704705D101680A6852080B4652001A6005
:101D0000012180F83D100020704702206870211DDD
:101D1000206800F0FAFA012028730121A970E87008
:101D200029716871A971E87129726872A972E872E3
:101D30006970002032BD38B5040001D1012032BDE8
:101D400000F0A4F818B900F0DCFA00F0ABFEDCE714
:101D500070B5044604F13E0009B902780FE0042989
:101D600008BF42780BD0082908BF827807D00C2919
:101D700008BFC27803D010290CBF02794279012A2A
:101D800001D0012070BD11B90222027014E00429B3
:101D900002D1022242700FE0082902D10222827091
:101DA0000AE00C2902D10222C27005E0102907BF07
:101DB00002220271022343712068012200F0C3FC59
:101DC00000F038F818BF904208D088421FBFDFF8F3
:101DD0009850A842DFF89460B04203D1456C45F4B6
:101DE000004545642068984218BFB0F1804F0BD081
:101DF00000F018F81CBF144DA84205D000F00FF8F1
:101E00001CBF9042884206D100F00FF818BFB0F511
:101E1000803F02D0206800F01FF8002070BD0B4BFF
:101E200098427047074B9842704781680D480840B8
:101E3000062870472068024B0649054A98427047B9
:101E4000002C01400004004000080040000C00404D
:101E500000340140004001400168024641F00101A8
:101E60001160704707000100004401400048014034
:101E700038B5040001D1012032BD00F007F818B9CF
:101E800000F03FFA00F069FDFFF73FBF04F13C05A9
:101E90006878704770B504000E4601D1012070BD0E
:101EA000FFF7F4FF18B900F02CFA00F0FCFD022057
:101EB0006870211D206800F028FA2068016821F070
:101EC00008010160012120680268164306600120B4
:101ED0002873A970E870297268726970002070BD5B
:101EE00070B504462068C5680669B10714D5AA070D
:101EF00012D56FF00201016101222277806910F092
:101F0000030F204602D000F0CFFD03E000F0CDFD2E
:101F100000F086F800202077700715D5690713D5E3
:101F200020686FF00402026102212177806910F4B9
:101F3000407F204602D000F0B7FD03E000F0B5FD81
:101F400000F06EF800202077300715D5290713D54B
:101F500020686FF00802026104212177C06910F047
:101F6000030F204602D000F09FFD03E000F09DFD2E
:101F700000F056F800202077F00615D5E90613D5B5
:101F800020686FF01002026108212177C06910F407
:101F9000407F204602D000F087FD03E000F085FD81
:101FA00000F03EF80020207706F0010105F0010066
:101FB000014206D020686FF001010161204600F067
:101FC000EEFD300608D5290606D522686FF08000A0
:101FD0001061204600F020FEF00508D5290606D540
:101FE00022686FF480701061204600F016FE7006C3
:101FF00008D5690606D522686FF0400010612046BA
:1020000000F00CFEB0060AD5A90608D522686FF0CC
:10201000200010612046BDE8704000F000BE70BD99
:10202000204600F0FDBDF8B500F005F901D1022011
:10203000F2BD012084F83C007AB9F3687268316817
:10204000206800F0F1FA2168886920F00C008861AE
:102050008A69B06802438A6163E0042A10D1F36898
:1020600072683168206800F034FB2068816921F4CF
:10207000406181618169B26841EA0221816150E079
:10208000082A24D12168F068726833681C311B0269
:102090004F68D1F804C02CF4807CC1F804C027F448
:1020A0002067D1F800C04FEA9C0C42EA8C0260F332
:1020B000071203F420630A603B434B60086820F07A
:1020C0000C0008600A68B06802430A6029E00C2A24
:1020D00026D12068F168726833681C301B0347689A
:1020E000D0F804C02CF4805CC0F804C027F420476A
:1020F000D0F800C02CF4407C4CEA022C61F30F3C79
:1021000003F42043C0F800C03B434360016821F45E
:10211000406101600268B16842EA0122026000E0A9
:10212000012500F001F8F2BD002084F83C002846AB
:10213000704770B500F07FF801D1022070BD01201A
:1021400084F83C0052B1042A19D0082A29D00C2A5C
:1021500038D0102A48D0142A57D068E0206800F000
:102160002FF92168886940F008008861886920F0AB
:10217000040088618A69306902438A6158E02068F6
:1021800000F060F92068816941F400618161816932
:1021900021F4806181618169326941EA02218161B2
:1021A00046E0206800F086F92168C86940F0080020
:1021B000C861C86920F00400C861CA693069024377
:1021C000CA6135E0206800F0B0F92068C16941F4C7
:1021D0000061C161C16921F48061C161C169326975
:1021E00041EA0221C16123E0206800F0C5F92168BD
:1021F000486D40F008004865486D20F004004865CF
:102200004A6D306902434A6512E0206800F0DEF949
:102210002068416D41F400614165416D21F48061A8
:102220004165416D326941EA0221416500E00125C5
:10223000FFF77AFF70BD0446002594F83C000128A2
:102240000E46704770B5064606F13C050024287816
:10225000012801D1022070BD0120287002226A707D
:10226000DFF81C043268936803409360086802003A
:1022700018BF102830D0202818BF30282CD0402874
:1022800026D0502819D060281BD0702806D0B0F571
:10229000805F27D0B0F5005F07D022E000F02CF877
:1022A0003068816841F0770105E000F025F830687A
:1022B000816841F48041816014E000F019F85021F8
:1022C0000BE0CA684968306800F019FA602104E040
:1022D00000F00EF8402100E00146306800F021FADD
:1022E00000E001240120687000F00BF870BD0000D0
:1022F000CA6849683068DDE1CB684A688968306837
:1023000017E200212970204670472DE9F043D0F8EC
:1023100000C0DFF87073DFF87033DFF87043DFF868
:102320007053DFF87063DFF87023DFF870E3DFF8D5
:102330007083B84218BFB0F1804F07D0404518BF36
:10234000704503D0904218BFB0420FD12CF07009F5
:10235000D1F804C04CEA090CB84218BFB0F1804F64
:102360000CD040451CBF7045904207D0B04218BF0A
:10237000A84203D0A04218BF984205D12CF4407265
:10238000D1F80CC04CEA020C4A692CF0800C42EAED
:102390000C0CC0F800C0B842D1F808C0C0F82CC07E
:1023A0000A68826218BFB04204D0A8421CBFA04293
:1023B000984201D10969016301224261BDE8F083BD
:1023C0002DE9F041066A026ADFF8B882DFF8BC72D4
:1023D000DFF8BCC2DFF8BCE252085200026226F00D
:1023E000020643688569DFF8BC220C6815402C435F
:1023F0008D683543DFF89062404518BF704504D0C2
:1024000060451CBFB842B0420DD1CA6825F008052E
:10241000154325F00405404518BF704505D06045BB
:1024200018BFB84201D0B04205D14A6923F44073C5
:102430001A438B69134343608461496841630562B1
:10244000BDE8F081F0B5036A026A974D22F01002F0
:10245000026223F02003446882690E6815408A688E
:1024600045EA062543EA021300F05BF818BF9042E4
:1024700008D1CF6823F0800343EA0713B04223F06A
:1024800040030AD090421CBF814A904205D07F4E43
:10249000B0421CBF7C4A904206D14E698A6924F43E
:1024A0004064164344EA8604446085614968816358
:1024B0000362F0BDF0B5036A026A22F48072026220
:1024C00023F400734468C669764A0D6816408A682A
:1024D000354343EA022300F024F818BF904208D1A4
:1024E000CF6823F4006343EA0723B04223F48063F8
:1024F0000AD090421CBF664A904205D0634EB0425B
:102500001CBF614A904206D14E698A6924F4405446
:10251000164344EA06144460C5614968C163036216
:10252000F0BD584E5B4AB042704770B5026A036A0C
:102530005D4C23F48053036222F400524368C56962
:1025400000F06BF842EA0532B0421CBF514DA84280
:1025500007D04F4EB0421FBF4C4DA8424A4EB0422A
:1025600004D14D6923F4804343EA85134360C46179
:1025700049680164026270BD70B5036A026A414E27
:1025800022F48032026223F400334468456D474AE6
:1025900015400A682A438D6843EA0543B0421CBFD0
:1025A0003C4DA84207D03A4EB0421FBF374DA8421B
:1025B000354EB04204D14D6924F4803444EA0524F8
:1025C0004460426549688165036270BD70B5026A06
:1025D000036A374C23F48013036222F40012436829
:1025E000456D00F01AF842EA0552B0421CBF294D71
:1025F000A84207D0264EB0421FBF244DA842224E0B
:10260000B04204D14D6923F4802343EA852343601B
:1026100044654968C165026270BD0E682C4044EA99
:1026200006248D68174E7047F0B5046A056A154E8A
:102630006D086D000562B042856918BFB0F1804F2A
:102640000DD0174EB0421CBF144FB84207D0124EE7
:10265000B0421FBF0F4FB8420D4EB04203D1AD087C
:1026600042EA850201E045F0010263F3071224F01B
:102670000A0401F00A01826121430162F0BD0000F9
:102680008800FEFF002C014000480140004401404A
:102690000040014000340140000C004000080040B0
:1026A000000400408CFFFEFFFF8CFFFE8FFFFEFF4B
:1026B000FF8FFFFE10B5036A046A640864000462B9
:1026C00023F00A03846924F0F00444EA02148461CC
:1026D00044E030B5046A056A25F010050562090179
:1026E000856925F4407545EA022563F30F3524F02A
:1026F000A00401F0A00185612143016230BD10B545
:10270000036A046A24F01004046223F0A0038469BD
:1027100024F4704444EA0234846143EA01130362FE
:1027200010BD826822F07002114341F00701816000
:10273000704710B5846824F47F442143114341EA73
:102740000321816010BD10B501F01F01036A01244F
:102750008C40A343036202FA01F1036A1943016248
:1027600010BD000018B587B004A800F047F868460F
:10277000002480E81E00DFF800434FF0FF304FF0E8
:102780008041E06021606260A2602261A261204617
:10279000FFF76EFB08B100F011FA002104910691D9
:1027A000204604A900F03EFA08B100F007FA002123
:1027B0000122009101920291039104226946204670
:1027C000FFF731FC08B100F0F9F908B010BD1FB5F2
:1027D00000F013F8A94CAA4921606260A2601F2191
:1027E000802200F029F808B100F0E8F920210091DA
:1027F000002202926946204618E068460021002225
:10280000002380E80E0070471FB5FFF7F6FF9D4CD0
:102810009D4921604F2060604FF6FF71A26000F07B
:102820000BF808B100F0CAF900F07BF800F0FAF9F3
:1028300008B100F0C3F91FBDE160A2612046FFF7B7
:10284000D1B918B599B00AA80021002200230024AC
:1028500080E81E0068468D4C80E80E001C2103A80D
:1028600000F06CFA2C210EA800F068FA884820606D
:10287000002140F28F10E0606160A16021610220C0
:1028800060618021A1612046FFF7ACF908B100F03A
:1028900095F94FF480500A900AA92046FFF7D2FC20
:1028A00008B100F08BF92046FFF745FA08B100F0B7
:1028B00085F908212046FFF7EDFA08B100F07EF90E
:1028C00000F02FF800F0AEF908B100F077F902221D
:1028D0000592C721049104220792602000210390F1
:1028E000069108910022099203A92046FFF721FCD6
:1028F00008B100F063F900204FF400510E900F90E2
:10290000109011901290139118900EA9204600F08B
:10291000C7F908B100F052F9204600F086F81AB065
:1029200010BD00210091029120466946704780B594
:102930005848594901604F2200234FF6FF71426009
:102940008360C160036143618361FFF74BF918B194
:10295000BDE8014000F032B901BD10B586B000F00D
:1029600086F82268B2F1804F1FD14C48C16841F00F
:102970000101C160C16801F0010100910099026884
:1029800042F0010202600221006800F001000090A4
:102990000098019102914FF0904000210391049121
:1029A0000121059101A900F0CDF906B010BD80B557
:1029B0000068334A3A49904207D1086840F0100055
:1029C0000860096801F0100109E02F4A904208D11F
:1029D000086840F020000860096801F020010091BB
:1029E0000AE02B4A904209D1886840F48030886020
:1029F000886800F480300090009801BD264A90421B
:102A000012D1886840F4003088600022886800F4A1
:102A1000003000900F210098192000F0B5FABDE8B1
:102A20000240192000F0CEBA01BD10B586B000F00A
:102A30001EF8226816498A4217D11848026842F0E7
:102A4000010202600421006800F0010000900222EF
:102A50000098019102920021039104914FF090405F
:102A60000E21059101A900F06DF906B010BD0446D4
:102A7000142101A800F062B9D43B0020203C0020C2
:102A8000001000406C3C002000140040B83C0020C6
:102A900000400140043D0020004401404C10024031
:102AA00058100240704770477047704780B500F07B
:102AB0009FFA00F03DF800F0F2FA3C483C494088AB
:102AC0004860C86100F026FB00F0B0FB00F0C6FBD8
:102AD00000F076FC00F08DFCFFF744FEFFF777FE78
:102AE000FFF792FEFFF7ADFEFFF721FF00F0E0FDDC
:102AF00000F0ACFE00F0F2FD00F097FF00F09BFF4D
:102B00002FA000F07CFF00BF0FF200120FF2F001C7
:102B100033A000F074FF7F21264800F0A1FF01F0F0
:102B200070F801F095F901F0E3F901F05BFAFEE7C6
:102B300080B596B0442105A800F000F9142168463C
:102B400000F0FCF84FF4007001F090FA08B100F0CA
:102B500035F84FF480310691012003211091059042
:102B60000222119014210F92129113921492159235
:102B700005A801F0B3FA08B100F020F80F200321F6
:102B8000009001910022029203920492042168466F
:102B900001F0F1FC08B100F011F817B000BD0068B9
:102BA0000549884208BF01F051BE704768140020F3
:102BB000D8140020B0390020002C014072B6FEE786
:102BC0004D6963726F20436C696D61746520537445
:102BD0006174696F6E2053656E736F722E0D0A00FB
:102BE00056657273696F6E20312E302E302042751B
:102BF000696C643A2025732025730D0A00000000DB
:102C000041756720203320323032340031363A317A
:102C1000343A313700000000704770477047704702
:102C200070470000F0B500F13C031A78012A01D189
:102C30000220F0BD01221A7002245C700568DFF8E2
:102C40005CC06E68AC683A4F654518BFBD4203D1A1
:102C500026F470024E6816430A6826F07006164382
:102C60006E600268624518BFB2F1804F0CD02E48EA
:102C700082421CBF2F4DAA4206D02A4882421EBF64
:102C8000BA422D4DAA4204D1886824F0800404433E
:102C900094600121597000201870F0BD002C014093
:102CA00030B590F83C20012A01D1022030BD01222C
:102CB00080F83C20CC688A684B681C4D24F4407432
:102CC000144324F480641C430A680B6924F40064F0
:102CD000144324F480541C434A698B6A24F400543E
:102CE000144324F4804423438A69046823F4702342
:102CF00043EA0243AC421CBF0D4A94420CD14A6ADB
:102D000023F4700343EA0253CA6923F08073134328
:102D100023F000750B6A2B436364002180F83C109C
:102D2000002030BD000C004000040040002C014099
:102D3000003401400008004000400140002201F042
:102D40008DBD00002DE9F84F0027784A784B4FF0F1
:102D50000F0805460E4636E0764CA54214BF0824FF
:102D600007248C40744944EA0E0441F82C40C143C6
:102D7000D2F808C0746801EA0C0CE40248BF40EACB
:102D80000C0CC2F808C0D2F80CC0746801EA0C0C34
:102D9000A40248BF40EA0C0CC2F80CC0D2F804C030
:102DA000746801EA0C0CA40348BF40EA0C0CC2F89A
:102DB00004C0D2F800C0746801EA0C01E40348BF03
:102DC000014311607F1C316831FA07F000F09E80EA
:102DD0000124BC4014EA0100F4D04FEA470C03215F
:102DE00001FA0CF16FEA010E716801F00309B9F103
:102DF000010F1CBF01F00301022912D1A968D6F806
:102E00000C900EEA010109FA0CF949EA0101A960E6
:102E1000696821EA04047168C1F30011B9400C43E8
:102E20006C60B900347904F00304032C21D0EC6801
:102E3000D6F808900EEA040409FA0CF949EA0404E9
:102E4000EC60347904F00304022C12D1FC0805EB89
:102E5000840401F01C09D4F820A008FA09FB2AEA2E
:102E60000B0AD6F810B00BFA09F949EA0A09C4F8B6
:102E700020902C680EEA040E347904F0030404FA5E
:102E80000CF444EA0E0CC5F800C0746814F4403F1A
:102E900098D0D3F800C0284C4CF0010CC3F800C007
:102EA0004FEA970CD3F800E00EF0010ECDF800E0E9
:102EB00001F00C01DDF800E054F82CE008FA01F410
:102EC0002EEA040EB5F1904F08BF00241DD01B4C14
:102ED000A54208BF012418D0194CA54208BF0224FE
:102EE00013D0184CA54208BF03240ED0164CA5429F
:102EF00008BF042409D0154CA54208BF052404D0FE
:102F0000134CA5427FF428AF06242AE7BDE8F18FD1
:102F10000AB18161704781627047426901EA020328
:102F2000914341EA03418161704700000004014080
:102F300060100240001C00480800014000040048E6
:102F400000080048000C0048001000480014004829
:102F5000001800480901020002D42048815470473B
:102F60001F4B02F00F021A4402F8041C70471D4B5D
:102F700019684FF6FF020002114000F4E0600843B8
:102F8000194908431860704770B5164B1C68C4F3A4
:102F900002230124C3F10705052D2EBF0F2504FAD6
:102FA00005F56D1E1E1D072E34BF0023DB1E2940B4
:102FB000994004FA03F3BDE870405B1E1A401143C8
:102FC000C8E70000010007D4012200F01F01074BF1
:102FD0008A40400943F820207047000000E400E0E8
:102FE00018ED00E00CED00E00000FA0500E100E063
:102FF000094810B5016841F4807101600320FFF7B2
:10300000B6FF0F2001F044FC0024002814BF012467
:1030100001F086FC204610BD0020024018B585B0A6
:1030200000230390049100930124019302946946C4
:1030300001A801F093FC50B1334C5C21204601F013
:1030400057FD411C222204F12C0000F0D8FC06B0F0
:1030500010BDF8B504460D461646002701E00834B9
:103060007F1CB74209D205EBC7002146D0E90023F7
:10307000002001F04BFD0028F1D0F1BD17B581B063
:1030800001F08BFD214C022201A92046FFF7E1FF50
:1030900001211F20FFF7C2FF022201A92DE0E0B5A8
:1030A00009216846FFF74AFE092218496846FEF7DB
:1030B00079F89DF80000552804BF9DF808001628EF
:1030C00006D1092269461248FEF76CF801200EBDB0
:1030D00000200EBD1FB509216846FFF72FFE01F045
:1030E0005CFD0A4C022269462046FFF7B2FF01212F
:1030F0001F20FFF793FF022269462046FFF7A9FF32
:1031000001F05BFD1FBD0000A492000800F800085C
:103110006814002070B586B014220021684601F0C2
:10312000A7FD3A483A4C01683A4D41F0040101606C
:1031300041F60806026802F0040205920599026849
:1031400042F080020260036803F080030593059952
:10315000026842F001020260036803F00103059374
:103160000599026842F002020260036803F002035C
:1031700005930599026842F0080202600022006887
:1031800000F0080005904EF2C03105982046FFF788
:10319000BFFE002231464FF09040FFF7B9FE0022FB
:1031A0002C212846FFF7B4FE4EF2C01100F034F88F
:1031B0002046FFF7C7FD0121019102220021039162
:1031C0000292009669464FF09040FFF7BBFD2C211C
:1031D00000F022F82846FFF7B5FD4FF4007100918A
:1031E0000122002102910391019269462046FFF7D6
:1031F000A9FD4FF4407000210090019102912846F2
:103200006946FFF79FFD06B070BD00004C100240FC
:1032100000080048000400480091012201920221A8
:1032200002910022039269467047000080B50A4867
:10323000016841F0010101600022006800F0010016
:103240000090052100980B20FFF79EFEBDE802408C
:103250000B20FFF7B7BE00BF4810024018B589B079
:103260000C22002106A801F003FD18220021684667
:1032700001F0FEFC4B4C4C482060002104206061B2
:103280006160002084F82000E160216121834FF417
:1032900080600121E062E16104F1300000224FF41E
:1032A000E861A260A162027042600272204601F0F1
:1032B00013FD08B1FFF782FC0020069006A9204606
:1032C00000F018FC08B1FFF779FC3849009106229C
:1032D0000192022102917F22039204210491002293
:1032E00005926946204601F051FE08B1FFF766FCE1
:1032F0000AB010BD30B5A9B004461422002101A8BF
:1033000001F0B6FC8C22002106A801F0B1FC206877
:103310002549884244D14FF480424FF040510692F3
:10332000259106A802F0E2F808B1FFF747FC204813
:10333000204D016841F400510160026802F400521E
:1033400000920099026842F00402026001210068C4
:1033500000F00400009003220098174801910292A7
:103360000021039101A9FFF7EDFC00216960E960EC
:10337000802129614FF4806110482860A9614FF4D1
:103380008070002268614FF44051AA60EA612962AE
:10339000284602F05DFB08B1FFF710FC2565AC6222
:1033A00029B030BDB03900200000045002003004C4
:1033B0004C100240503D0020000800480800024028
:1033C00080B5AE48AE49AF4A016042600021C1609D
:1033D0004FF080530C214161836000220021026183
:1033E000826101624262002302F08DFC00B116E0AE
:1033F00001BD80B5A448A54901604FF4E132002326
:103400000C2142608360C360036141618361C361D9
:103410000362436202F0BEFC00B100E001BDBDE802
:103420000140FFF7CBBB10B5994C9A496060216011
:103430000020A060E06020610C21A061E0612062BA
:1034400060626161204602F0A5FC14E010B5924C68
:103450009249216060600C2161610020A060E06001
:103460002061A06100212062E161616200230022ED
:10347000204602F048FC08B1FFF7A0FB04F18801E8
:103480002046BDE81040012202F018BD30B5A9B0B9
:10349000044614220021684601F0EAFB8C22002138
:1034A00006A801F0E5FB206875497D4C884222D1D1
:1034B00020224FF480610692199100F0C2F808B101
:1034C000FFF77CFB206940F001002061206900F0DB
:1034D000010005900598216841F00201216040F645
:1034E0000241226802F002020592022205986D480C
:1034F00000F0AAF838E065496B4D884237D11022B8
:1035000000210692189100F09CF808B1FFF756FBD5
:10351000E06840F48010E060E06800F480100590FE
:1035200000F082F8226802F00402059205982168F2
:1035300041F0080121604FF48051226802F0080236
:1035400005920222059800F07FF82846FFF7FAFB63
:103550000221019100220420029203210090039194
:103560000822049269465148FFF7ECFB5AE04949AA
:1035700088421ED101220692149200F062F808B12E
:10358000FFF71CFB606940F480406061606900F4F3
:10359000804000F04FF84FF4C061226802F0010251
:1035A00000F05CF8002205212520FFF7EDFC252026
:1035B00036E03A49884235D104221021069216910C
:1035C00000F03FF808B1FFF7F9FAE06840F4802016
:1035D000E060E06800F4802000F02CF8226802F03F
:1035E0000102059200F020F84FF40041226802F039
:1035F000040200F033F802210191002202924FF4FC
:1036000040600321009003910722049269462846F6
:10361000FFF798FB002205212720FFF7B5FC2720A4
:10362000FFF7D0FC29B030BD0598216841F00401B6
:103630002160704705900598216841F001012160E3
:10364000704706A801F052BF00910192002102913B
:1036500003220821049103926946704705920222D1
:103660000598009101920021029103220721049103
:10367000039269464FF09040FFF764BBA0380020EA
:10368000008000402433030028390020005000400F
:1036900088370020003801401438002000480040DE
:1036A0004C1002400004004800080048000C00488C
:1036B00010B55F4C5F4800F027F808B1FFF77EFABD
:1036C0000021204603F0F4F808B1FFF777FA002153
:1036D000204603F002F900B125E010BD10B5564CAC
:1036E000564800F011F808B1FFF768FA00212046AB
:1036F00003F0DEF808B1FFF761FA0021204603F07D
:10370000ECF800B10FE010BD4D492060002201200F
:10371000E0606160A26022616261A261E261226296
:10372000204603F005B9BDE81040FFF747BA30B5B1
:10373000A9B0044614220021684601F099FA8C22AF
:10374000002106A801F094FA20683A493D4C3E4D0C
:10375000884221D140224FF4805106921A9106A846
:1037600001F0C4FE08B1FFF729FA286840F0020012
:1037700028601222296801F002010591C02100F0A1
:103780004BF82046FFF7DEFAE86840F40010E860E6
:10379000E86800F400103BE0284988423AD14FF431
:1037A0008072002106921C9106A801F09FFE08B1CC
:1037B000FFF704FA286840F001002860296801F04A
:1037C000010105910598296841F0020129608021D5
:1037D0002A6802F002020592122200F01DF84FF052
:1037E0009040FFF7AFFA12210191002202921020BF
:1037F0000321009003910422049269462046FFF7BA
:10380000A1FAE86840F40000E860E86800F400000D
:103810000090009829B030BD0598009101920021D8
:10382000029103220421049103926946704700002B
:10383000E03A002000540040343B0020005C00408F
:10384000EC9C9010000400484C10024080B52848C1
:10385000284901604FF482724FF44071C1604260A8
:103860000721C16200234FF4802208218360036195
:1038700043618261C36103624362836203634163A4
:1038800003F036FB18B1BDE80140FFF797B901BD61
:1038900010B586B004461422002101A801F0E8F911
:1038A00021681448814221D11348C16841F4804104
:1038B000C160C16801F4804100910099026842F042
:1038C000020202604FF47041006800F002000090B4
:1038D00002220098094801910292002103910322DB
:1038E00005210591049201A9FFF72CFA06B010BD3D
:1038F000183A0020003800404C10024000040048F4
:1039000070B5524D6B7806460024B34214D1285D41
:1039100080B92819083003F05BFB2819012E406894
:1039200002D1FFF780FD03E0032E08BFFFF78EFDF5
:1039300001202855281970BD687E1824B042E6D0B1
:10394000002070BD02B500281CBF0178002912D0EC
:103950004078012804D10A23012269463C4805E049
:10396000032808D10A23012269463A4802F056FA90
:1039700008B9012002BD002002BD38B504460D463D
:1039800006E00D2100F01BF80A2100F018F86D1C6C
:10399000287830B10A28F4D015F8011B00F00FF890
:1039A000F6E731BDF8B504460D461646002703E09C
:1039B000E95D00F004F87F1CB742F9DBF1BD204659
:1039C000C0E700281CBF017800291EBF01694069BB
:1039D000814201D001207047002070471CB50021B2
:1039E0008DF800100446FFF7ECFF20B1694604F1A2
:1039F000080003F00CFBFFE79DF8000016BD0EB4B5
:103A000078B5154D044605F1CC0664213046FFF724
:103A100095F905AA2146304603F012FB2868314685
:103A2000FFF7ABFF71BC5DF810FB10B50A4CC82264
:103A3000211D012005E010B5084C4FF49672211DA0
:103A40000320FFF75DFF206010BD0000D8140020A8
:103A50008837002014380020003400203035002042
:103A60007CB50446002004F154060D4600903178E0
:103A7000012901D1022076BD0120307000F035F817
:103A8000010070682AD120F4885040F00200706074
:103A900005F080452268DFF85800936803401D4315
:103AA00045F00045956020688068C00F10D00098F0
:103AB000401C00900098B0F5912FF4D3706820F06E
:103AC000020040F01000706000203070012076BDD0
:103AD0007268012060F30102726002E040F01000A1
:103AE000706000203070084676BD204601F064BC4E
:103AF000C0FFFF3F2DE9F04100F154049AB0237854
:103B00000022012B08BF022052D00125257000267B
:103B10001696002517950368294DAB422CD1294FE5
:103B2000DFF8A4E03B68DEF800506D073AD45B078D
:103B300038D40B68254DDFF898C0264E0BB3D6F865
:103B400000804B6890F8300028F4604843EA08038E
:103B500043EA4038C6F80080DEF800003B68DCF835
:103B6000007018433843C3071FD437680868896852
:103B70003D4005430D4313E000F01DF82270012085
:103B800016E0306820F460403060DEF800003968EC
:103B9000DCF8003008431843C00706D431680D40F4
:103BA000356002E000F007F8012200202070104686
:103BB0001AB0BDE8F081606840F020006060704796
:103BC000000004500801045008000450E0F0FFFF1A
:103BD000080204500803045010B50023DAB2825CD6
:103BE0005140C9B208224C0009064CBF84F0310193
:103BF0002146521EF7D15B1CDAB2022AEEDBC8B2B4
:103C000010BD1FB50122202189488A4CFFF780F999
:103C1000012003F02FFA02A903A800F083F850B99D
:103C20005C21204600F064FF411C512204F1300069
:103C3000FFF7E5FE0DE0029803F030FACDE9000150
:103C4000039803F02BFA02460B4604F19800FFF7A5
:103C5000D6FE002004B010BD0FB47FB5062102A827
:103C6000FFF76CF8BDF844109DF84040724D01AA72
:103C7000002010800B0A8DF804308DF805104FF6E7
:103C8000FF76009602232146284602F0ADFE0096FC
:103C9000062302AA2146284602F008FF80B9FF2128
:103CA00002A8FFF799FF02ACA17888420AD0FF2151
:103CB0000DF10B00FFF790FF9DF80D10884201D029
:103CC000012022E09DF8082063781298139943EAB6
:103CD000022300EE103A00F01DF89FED4E1ADFEDC2
:103CE0004E1A40EE811AC0ED001AE0789DF80C20C3
:103CF00042EA002200EE102A00F00CF89FED471A6D
:103D000020EE811A81ED001A002004B070BC5DF82D
:103D100014FB0000B8EE400ADFED410AC0EE200AB5
:103D2000704700002DE9F843C4B004460D46DFF8A3
:103D30000C9126A849467822FDF734FA08A809F123
:103D400078017822FDF72EFA0027DFF8F48008A822
:103D500000EB8700079026AE06EB8700069084B044
:103D6000414668462822FDF71DFA0FBCFFF774FF95
:103D700030B9012000F06AF97F1C0A2FE7DB08E068
:103D80002C485C2100F0B4FE411C842209F1F000B3
:103D900033E002220A2126A803F0A4F901900222AE
:103DA0000A2108A803F09EF99DED010A0090DFEDBD
:103DB0001D0A00F047F81F4804DBDFED1B0A00F086
:103DC00041F807D45C2100F093FE411C8B2209F5D9
:103DD0009A7012E09DED000AB5EE400AF1EE10FA7D
:103DE00004DBDFED120A00F02DF80AD45C2100F0AC
:103DF0007FFE411C8C2209F5D670FFF700FE0020E3
:103E000004E00198206001200099296045B0BDE8D8
:103E1000F083000000002F43000034C20000C842BD
:103E200000FF7F47000020C20100AA420100C842F3
:103E30000004004880910008E03A0020908E0008BD
:103E400080140020B4EE600AF1EE10FA7047000012
:103E5000E0B500BF20A000788DF80400FF2100919C
:103E6000012301AAEE21194802F0BEFD07BD0000A2
:103E70003EB500BF19A0154C00788DF80400FF2551
:103E80000095012301AAEE21204602F0ADFDFF209E
:103E9000009003230E4D2A46EE21204602F006FE36
:103EA000287869780B4A41EA0021A87840EA012085
:103EB000642190FBF1F100EE101A85ED010AB8EED5
:103EC000C00A10EE100A106237BD0000343B00201B
:103ED000583E0020D43D0020480000003000000083
:103EE0001C4B036003F1540008608021116070478F
:103EF00010B500211CA0184C00F079F8A06000213A
:103F000020A000F074F860605FF0000124A000F0D1
:103F10006EF820605FF0000128A000F068F8E06013
:103F200010BD38B50D4C0E4D286803F008FB206815
:103F300003F005FB642000F089F8F5E780B54FF445
:103F40007A7000F083F84FF400710648FEF7E5FF41
:103F5000F5E70000AC3100203C3E0020003400209A
:103F6000303500200008004840940008233F000836
:103F7000020000000000000000010000000000003E
:103F800000000000589400083D3F0008FDFF0000BD
:103F90000000000020000000000000000000000001
:103FA0004C94000825840008030000000000000075
:103FB0008000000000000000000000001C940008C9
:103FC000C38700080100000000000000800000001E
:103FD000000000000000000001460020842918BFF6
:103FE000C81C704780B503F024FC002002BD38B522
:103FF000044684B060690D4600281CBFA0690028F3
:1040000012D0B4F90800FFF7E7FFA16902912B462F
:1040100062690192009022692168606803F0FEFAEB
:104020000390039805B030BDB4F90800FFF7D4FF42
:1040300003A9019100902B4622692168606892B221
:1040400003F01DFB0128ECD00020EBE780B519211F
:10405000B0FBF1F000B9012003F0D1FB002002BD5C
:10406000DFF86C00006800F4C060704710B5DFF83E
:104070006010B0F5007F086800F4C0601DD1B0F595
:10408000007F22D00A68DFF84C30012060F34A221A
:104090000A6032201C68DFF840204443B4FBF2F091
:1040A000401C00E0401E4A69530501D50028F9D1A3
:1040B0004869410509D5032010BDB0F5806F04D0D3
:1040C0000A68022060F34A220A60002010BD000046
:1040D00000700040D414002040420F002DE9FC473E
:1040E000050066D0DFF82477DFF83067BC68D7F8C2
:1040F0000C802878C10604F00C0408F0030848D5A9
:1041000024B10C2C08BFB8F1010F2CD138688107FD
:1041100002D5A86900284CD0396808074EBF396815
:1041200071680909286A01F0F001814206D200F0A5
:1041300032FB00283DD100F006FA07E000F003FA58
:1041400024B9286A00F027FB002832D100F0ABFA2E
:10415000BA6800F097FADFF8BC06006800F098FB38
:10416000010016D0E9E1A86928B3396841F00101DE
:10417000396003F01DFD81463868810707D403F0DC
:1041800017FDA0EB09000328F6D30320D5E100F0CA
:10419000DAF92878C10755D5082C04D00C2C08BFB3
:1041A000B8F1030F17D1386881034BD56868002830
:1041B00048D10120C1E138684008400000F0D8F93A
:1041C000814638688107E4D503F0F2FCA0EB0900D2
:1041D0000328F6D3D9E76868B0F5803F04D1386882
:1041E00040F48030386011E0B0F5A02F386806D177
:1041F00040F480203860396841F4803105E020F4D3
:1042000080303860396821F480213960686860B195
:1042100003F0CEFC81463868810313D403F0C8FC58
:10422000A0EB09006528F6D3AFE703F0C1FC814697
:104230003868810306D503F0BBFCA0EB09006528B4
:10424000F6D3A2E72878810713D5042C04D00C2CD0
:1042500008BFB8F1020F22D13868410502D5E868DD
:104260000028A6D07868296920F0FE4040EA016065
:1042700078602878010742D56869002870682FD0D7
:1042800040F00100706003F093FC80467068810785
:1042900035D403F08DFC00F052F9F7D375E7E868E8
:1042A00078B1396841F48071396003F081FC80464F
:1042B00038684105D6D403F07BFC00F040F9F7D311
:1042C00063E7386820F4807000F052F9804638685F
:1042D0004105CED503F06CFC00F031F9F7D354E77B
:1042E00040084000706003F063FC804670688107FE
:1042F00005D503F05DFC00F022F9F7D345E72878F7
:10430000410767D5B86DC1004FF000080AD4B86DF9
:1043100040F08050B8654FF00108B86D00F0805053
:1043200000900098DFF8F894D9F80000C10513D484
:10433000D9F8000040F48070C9F8000003F038FCA0
:104340008246D9F80000C10506D403F031FCA0EB89
:104350000A000328F5D318E7A868012804D13068BB
:1043600040F00100306010E00528306806D140F0D0
:1043700004003060316841F0010105E04008400070
:104380003060316821F004013160A86841F2893958
:1043900060B103F00DFC82463068810713D403F04E
:1043A00007FCA0EB0A004845F6D3EEE603F000FC5C
:1043B00082463068810706D503F0FAFBA0EB0A00BD
:1043C0004845F6D3E1E6B8F1000F03D0B86D20F010
:1043D0008050B8652878810621D5686A0028B068C1
:1043E0000ED040F00100B06003F0E2FB8046B06800
:1043F000810714D403F0DCFB00F0A1F8F7D3C4E686
:1044000040084000B06003F0D3FB8046B0688107ED
:1044100005D503F0CDFB00F092F8F7D3B5E6A86A16
:10442000002800F08980022872D1F868EA6A00F05A
:104430000301914201BF00F0700110312A6BB1EB12
:10444000021F1DD16A6B00F4FE41B1EB022F02BFC7
:1044500000F07841AA6BB1EBC26F11D1EA6B00F4A6
:10446000C00101F500115208B1EB425F08D1296C7F
:1044700000F0C06000F100704908B0EB416F43D01C
:104480000C2C46D03868410101D43868C1003FF592
:1044900090AE00F06AF804463868810105D503F053
:1044A00087FB001B0328F7D36FE6F868DFF8741367
:1044B000EA6A0840296B1043491E40EA0110EA6B82
:1044C000696B520840EA0120296C521E490840EAF3
:1044D0004250491E40EA4160A96B40EAC160F86061
:1044E000386840F080703860F96841F08071F96098
:1044F00003F05EFB0446386881011DD403F058FBCD
:10450000001B0328F7D340E63868810114D4E7E79D
:104510000C2C3FF44EAE00F028F8044638688101B8
:1045200005D503F045FB001B0328F7D32DE6F868FB
:10453000DFF8F4120840F8600020BDE8F687A0EB31
:10454000080003287047386840F008003860396870
:10455000286A21F0F001014339607968E86921F4A3
:104560007F4141EA002179607047386820F080700F
:10457000386003F01DBB2DE9F0410400884655D09A
:10458000DFF8A862306800F00700404502D200F072
:104590006FF84BD12078DFF87452810706D5A068F8
:1045A000A96801F0F001814200F076F82078C10797
:1045B0002AD56068032802D129688A0108E0022808
:1045C00002D129688A0303E00028296802D18A07FA
:1045D00002D42BE04A0529D5A968890840EA810060
:1045E000A86003F0E5FA0746A868616800F00C00CF
:1045F000B0EB810F08D003F0DBFAC01B41F2893128
:104600008842F1D3032031E02078810706D5A068E5
:10461000A96801F0F001884200F03EF8306800F02F
:104620000700804504D200F023F801D001201DE0EE
:104630002078410705D5AA68E06822F4E0620243C9
:10464000AA602178080706D5A968206921F460517D
:1046500041EAC001A96000F026F8AA6800F012F84B
:10466000BDE8F0416B48006800F012B9BDE8F08188
:104670003168C90848EAC1013160306800F00700BC
:10468000404570476A49C2F30312895C604A01F0F1
:104690001F01C8401060704704D2A96821F0F001E2
:1046A0000843A860704770B5584A634B9068D66855
:1046B0000025002110F00C0006F003065F4C03D02B
:1046C0000C2812D1012E1AD115682E0704D4524D90
:1046D0002E68C6F3032502E01568C5F30315584E8E
:1046E00056F8255048B9294624E0042808BF214639
:1046F00020D008281ED119461CE00C281AD1D068F9
:1047000000F00300022803D0032808BF1D4600E084
:104710002546D168D068D268C0F306204543C1F36E
:104720000210C2F34161401C491CB5FBF0F0490086
:10473000B0FBF1F1084670BD35483E4A0068136889
:104740004049C3F3022206E031483A4A0068136840
:104750003C49C3F3C222895C01F01F01C840704785
:1047600010B50F220260334A136803F0030343605D
:10477000146804F0F0048460136803F4E063C36019
:104780001268D20802F4E06202612848026802F06E
:1047900007020A6010BD7CB52B4E05463068002428
:1047A000C10002D5FFF75CFC0EE0306840F080509D
:1047B0003060316801F0805100910098FFF750FCA3
:1047C000316821F080513160B0F5007F04D1802D37
:1047D0000CD9A12D09D304E0802D88BF032405D86E
:1047E00001D1022402E0702D00D101240F4801689C
:1047F000C90844EAC1010160006800F00700A04256
:1048000001D0012076BD002076BD000000100240DE
:10481000D4140020B01400209410024090100240E4
:10482000007000408C809D01FCFFEEFE00200240E5
:10483000949200080810024000127A000024F4004C
:104840003093000860940008581002400248416804
:1048500002788A1842607047A814002000B500BF93
:10486000130096469446103928BFA0E80C50FAD899
:104870005FEA417C28BF0CC048BF40F8042BC90741
:1048800028BF20F8022B48BF00F8012B00BD000014
:1048900078B504461D481E4D87B0016841F400619B
:1048A000016001A9006800F40060009002A8009A6D
:1048B000FFF756FFFFF748FF1649174B2960B0FB7B
:1048C000F3F0401E40F2E73268600021EA6029619F
:1048D000A960A9612846FDF785F9060012D128468E
:1048E000FDF7CDF906000DD11920FEF76BFB102C5A
:1048F00007D2002221461920FEF746FB0748046034
:1049000000E00126304608B070BD00006010024093
:10491000883B0020002C014040420F00B0140020D2
:104920000D4882B0816841F001018160816801F029
:10493000010100910099026842F080520260002259
:10494000006800F0805000900F2100986FF0010087
:1049500002B0FEF719BB00BF581002402DE9F04726
:10496000DFF87841054620788946012808BF0220F3
:1049700057D0012020704CF2503800F054F85FEA14
:10498000000A4BD10020DFF858616060316888056B
:104990000AD53168480505D5316821F48061316058
:1049A00003200CE0012107E03068410506D530689E
:1049B00020F4806030600221217701E00020207720
:1049C000296801290BD1686800F030F800F02BF855
:1049D00082467169DFF80C01014071611CE04FF003
:1049E000FF31C9F80010AF6800E07F1CA868E968D3
:1049F0000818874210D26968384600F029F800F09C
:104A000012F882467069DFF8E01008405FEA0A0297
:104A10007061EAD0C9F8007000F033F8002020700F
:104A20005046BDE8F087404600F0CFB8C2072F4996
:104A300003D50B6843F004030B60800703D50A68B5
:104A400042F400420A60086840F480300860704711
:104A5000C907264A04D5136823F40063136003E0F2
:104A6000116841F400611160116860F3CA011160BE
:104A7000106840F002001060116841F4803111604C
:104A8000704710B51548164A017F012918BF032940
:104A90000FD1136823F400731360146844F40064A6
:104AA0001460136823F400631360146844F4007402
:104AB0001460022918BF03290BD1116841F48051F9
:104AC0001160136823F480531360116841F480610E
:104AD00011600022027710BD00000000B414002015
:104AE00000200240FB7FFFFF05F8FFFF142002407B
:104AF0000246C9B2002013788B4205D012F801CBD0
:104B0000BCF1000FF7D170471046F7E72DE9F84FD9
:104B1000504F0546387800268A4690469946012827
:104B200008BF022037D0012038704CF2503000F01E
:104B30004CF8834660BB484C78602168480506D530
:104B4000216821F4806121600220387701E0002192
:104B50003977504642464B461DB900F05CF80126B5
:104B60000AE0012D18BF022D06D1114600F05FF8B2
:104B7000022D08BF4FF480264CF2503000F025F88B
:104B800083461EB1606920EA06066661FFF779FF79
:104B9000002038705846BDE8F28F3149CA680020BD
:104BA000002A00D4704710B52E4A2F4C0A600C60C2
:104BB000C968002948BF012010BD2C48016841F098
:104BC0000041FFE701600020704770B5054602F024
:104BD000EFFF0646214C2068C10309D515F1010FEE
:104BE000F9D002F0E5FF801BA842F4D3032070BD8A
:104BF00021684CF2FA30084006D016494A68024350
:104C00004A602060012070BD2068C10744BF0120B8
:104C10002060002070BD10B514490C6844F00104F8
:104C20000C6040F8042BBFF36F8F036010BD10B50C
:104C30000E4A136843F480231360EFF3108372B6B7
:104C4000402251F8044B40F8044B521EF9D183F333
:104C5000108810BDB4140020002002401020024033
:104C60000820024023016745AB89EFCD14200240A4
:104C700010B5044610460A460146204602F09EFF43
:104C8000204610BD603000EB8100006800F0F84065
:104C90007047603000EB8100016821F000410A4359
:104CA00002607047C06800F44060401E8041C00F41
:104CB000704700F11403C80D10B500F00400C018CF
:104CC000090D01F01F01036807248C40A34302FA79
:104CD00001F11943016010BDF8B50446002000251C
:104CE00000900CB90120F2BD04F15406706828B997
:104CF0002046FEF7FFFA0020B06030702168886817
:104D0000800004D58A68DFF85C0202408A6021686E
:104D10008868C00012D48A68DFF84C02024042F072
:104D200080528A60DFF84412DFF844220868B0FB42
:104D3000F2F2521C5200009200F036FB20688168AB
:104D4000C90008D4726842F0100272600125B1688F
:104D500041F00101B160816872688908D30600D40E
:104D6000CA0700F18180736823F4807343F0020363
:104D700073608068C00714D4DFF8F821DFF8F831D9
:104D800010681A68DFF8F4713B6810431843C007D5
:104D900007D4DFF8EC211368606823F47C13034325
:104DA000136004F13002607E536894F8207043EA87
:104DB0004033E0681843A3680343012F43EA0743E5
:104DC00003D1606A401E43EA4043A06A20B100F468
:104DD00070701843E36A03432768DFF8A801D7F827
:104DE0000CC000EA0C000343FB60C9072368986805
:104DF00026D4000724D4DF68DFF88C11D0690F4077
:104E0000217E0743107847EA813747EA4007DF6091
:104E1000107A01280FD123681F69D16810696FF3D8
:104E20008A070F435169074390690F43074347F0CF
:104E300001071F6104E02068016949084900016118
:104E4000206901282068016B05D1E2690909521E19
:104E500042EA011101E009090901016301207168B9
:104E600060F30101716004E0706840F01000706050
:104E700001252846F2BD0646DFF8040104687047A4
:104E80002DE9F04105460E46FFF7F6FF28688168D8
:104E90004907904604F01F0461D405F154073A789D
:104EA000012A5CD00121DFF888253970904218BFB3
:104EB000002C03D0052C18BF092C4CD1284600F03B
:104EC00029FA010044D17968DFF86005014041F416
:104ED00080717960DFF8DC032968814200D11CB958
:104EE000786820F4801078607868C10446BFB8689C
:104EF00020F006000020B8604346286D0FF2615193
:104F0000C162286D0FF2C5510163286D0FF2C551C2
:104F100041631C212A6811600020387032462868DD
:104F2000416841F0100141602868C16841F0010109
:104F3000C160286800F14001286D00F0EDFD2A688D
:104F4000DFF8F01493680B4043F00403936007E02C
:104F50000021397004E0002201203A7000E00220B4
:104F6000BDE8F081C0FFFF5FC0FFFF7FD4140020C9
:104F7000400D0300080004500801045008020450CA
:104F80000803045007C0F0FFF9BFFFFFF8B506465D
:104F9000002006F154050F460090002429780129CD
:104FA00001D10220F2BD01202870306881684907D4
:104FB00000F175817968062910D2891E03290CD861
:104FC000DFE801F0020406080C2107E0122105E0E9
:104FD000182103E04FF4807100E0062100F1300356
:104FE000880900F00C003A68C01801F01F0103683E
:104FF0004FF01F0C0CFA01FCC2F3846223EA0C038D
:1050000002FA01F119430160306882688168520731
:1050100031D409072FD4BA68B2F1004F08D13968EA
:105020000022FFF746FE3068416941F0004106E08A
:105030003968FFF73EFE3068416921F00041416167
:105040003068C1683A69042A16D060303B6800EBCA
:10505000820C9748DCF80020024003F0F843134329
:10506000C9087A69480000F006008240134343F003
:105070000043CCF8003076E00021FFF703FE400348
:105080003068214604D1FFF7FDFDC0F3846003E0E2
:10509000FFF7F8FD00F01BF939684A030EBFC1F3B2
:1050A000846191FAA1F1B1FA81F1884204D13068AA
:1050B00000220021FFF7EDFD00F016F9400304D1B6
:1050C00000F012F9C0F3846003E000F00DF900F085
:1050D000FEF839684A030EBFC1F3846191FAA1F169
:1050E000B1FA81F1884204D1306800220121FFF732
:1050F000D0FD00F0F5F8400304D100F0F1F8C0F362
:10510000846003E000F0ECF800F0E1F839684A034D
:105110000EBFC1F3846191FAA1F1B1FA81F1884225
:1051200004D1306800220221FFF7B3FD00F0D4F86B
:10513000400304D100F0D0F8C0F3846003E000F035
:10514000CBF800F0C4F839684A030EBFC1F384619C
:1051500091FAA1F1B1FA81F1884204D130680022BC
:105160000321FFF796FD31688868C00747D4FA68C5
:105170003B68D1F8B0C0DFF8C0E202F01802C3F318
:1051800012002EFA02F22CEA000013400343C1F889
:10519000B030F868DFF8A412884230D13868410393
:1051A0000EBFC0F3846290FAA0F1B1FA81F2521CF2
:1051B000012102F01F020A2A0DD200F099F892068E
:1051C00003F01F03401C02F0F842994000F01F005A
:1051D00000F072F80FE000F08BF8401C920603F02C
:1051E0001F0300F01F0002F0F84299400A3800F057
:1051F00063F841F00071BA683068FFF75AFD3B6808
:10520000DFF83C0203424FD0DFF83802DFF838C243
:105210000168DFF81C72DFF83422634501F0E071A9
:105220001ED10B0240D43368934218BFBB423BD11E
:1052300000F048F841F400010160DFF81402DFF8E3
:1052400014220168B1FBF2F2521C0C20424300927E
:10525000009800281EBF0098401E0090F8D123E05F
:10526000DFF8F4E173450BD1CB011DD433689342D1
:1052700018BFBB4218D100F025F841F080710CE056
:10528000DFF8D871BB420FD14B020DD4366896427D
:105290000AD100F017F841F48001016004E0686869
:1052A00040F0200068600124002028702046F2BDF4
:1052B00000F0FF0300010450114300EB400041EAFD
:1052C00000517047026822F0E0721143704790FA73
:1052D000A0F0B0FA80F0704730680321FFF7D2BC2D
:1052E00030680221FFF7CEBC30680121FFF7CABC4D
:1052F000420306D1C0F38462C0F38463C0F38460C8
:1053000005E090FAA0F0B0FA80F213461046521C65
:105310005B1C70477CB504460020009021688868BB
:10532000C20735D488686FF39E1000282DD1886895
:10533000404D284040F00100886042490868000262
:105340000AD54349434B0A68B2FBF3F35B1C0C20BC
:105350004343009300F028F802F02AFC0646206838
:105360000168CA0714D48068C00705D42068816822
:10537000294041F00101816002F01AFC801B0328E2
:10538000EDD320680168CA07E9D400F003F876BDC0
:10539000002076BDA06D40F01000A065E06D40F0EB
:1053A0000100E0650120704702E00098401E009077
:1053B00000980028F9D1704738B5044621688868FC
:1053C0008A68D2072ED580072CD48A6802F00D0295
:1053D000012A1DD18A681748024042F002028A6001
:1053E00003212068016002F0E3FB0546216888681C
:1053F000C10717D502F0DCFB401B0328F6D3206859
:105400008168C807F2D5A16D41F01001A16503E0E4
:10541000A06D40F01000A065E06D40F00100E06577
:10542000012032BD002032BD00000000FEF1FFFF70
:1054300000020450C0FFFF7FFFFF070000007F4015
:105440000000088008030450000052C70000045008
:10545000D4140020400D0300000084CB0100008024
:1054600010B5846AA16D11F0500F22D1A06D40F4E7
:105470000070A065216808680207084606D5FFF796
:1054800011FC88B12068C168880401E0C168880700
:105490000AD4A16D21F48071A165A06DC10403D46B
:1054A000A06D40F00100A0652046BDE8104002F06C
:1054B0008EBBA16DCA0604D52046BDE8104002F09F
:1054C00087BB216D4A6BBDE810401047806A02F02F
:1054D00080BB0000806A816D41F040018165C16D33
:1054E00041F00401C16502F073BB00002DE9F84FE3
:1054F000064600253068DFF850730105A84621D51F
:10550000B06E70B1B0F5800F17D0B0F5000F03D0BA
:10551000B0F5400F09D013E03A6842F480323A60A7
:1055200004E0002100F08DF9054655B9F96FB06E21
:1055300021F440010143F96704E000F07CF9F3E74E
:105540000125A8463068C10421D5F06EA8B1B0F19C
:10555000807F17D0B0F1007F03D0B0F1407F04D03E
:1055600013E0396841F4803139607DB9F96FF06E2C
:1055700021F040710143F96709E0002100F061F971
:105580000546F2E700F057F9FAE70125A84630682A
:10559000DFF8B84281032ED5F86CC1004FF0000946
:1055A0000AD4F86C40F08050F8644FF00109F86CB0
:1055B00000F0805000900098DFF894A2DAF8000024
:1055C00040F48070CAF8000002F0F2FA8346DAF87C
:1055D0000000C10500F18B8002F0EAFAA0EB0B009D
:1055E0000328F4D30325A846B9F1000F03D0F86CC3
:1055F00020F08050F8643078C10705D5FA6FB06BA1
:10560000920840EA8202FA673178880705D5F96F77
:10561000F06B21F00C010143F9673178480705D59B
:10562000F96F306C21F030010143F96731780807D8
:1056300005D5F96F706C21F0C0010143F96731782D
:10564000C80605D5F96FB06C21F440710143F967C4
:105650003178880605D5F96FF06C21F4406101437B
:10566000F9673168880505D5F96F306E21F440215E
:105670000143F9673168480505D5F96F706E21F46B
:1056800040110143F9673178480605D5F96F306D4F
:1056900021F440510143F9673178080605D5F96FC7
:1056A000706D21F440410143F9673168C80505D5A3
:1056B000F96FB06D21F440310143F9673168C802D8
:1056C00005D5E168F06D890840EA8101E160316843
:1056D000880447D5F96F306F21F040610143F967C5
:1056E000306FB0F1006F35D100F0A0F83AE0002D36
:1056F0007FF479AF206810F440701EBF06F184017A
:105700004A6890420BD02068216841F480312160C2
:1057100020F44070226822F4803222602060C007AA
:105720000FD502F045FA05462068810709D402F03A
:105730003FFA401B41F289318842F5D34FF003080C
:1057400052E706F184022168506821F44071014358
:10575000216049E7B0F1806F04D100F071F80100D9
:1057600018BF80463068010314D5FA6F706F22F0BD
:1057700040620243FA67706FB0F1006F02D100F02F
:1057800055F807E0B0F1806F04D100F059F801003E
:1057900018BF80463068410314D5FA6FB06F22F00D
:1057A00040620243FA67B06FB0F1006F02D100F0BF
:1057B0003DF807E0B0F1806F04D100F041F801003E
:1057C00018BF80463068410418D5FA6FF06F22F098
:1057D00040520243FA67F06FB0F1805F03D10221BB
:1057E00000F02FF807E0B0F1005F07D1022106F1C9
:1057F000200000F0A2F8010018BF804630680104C4
:1058000006D5FA6FD6F8800022F080420243FA678C
:105810003168C80306D5F96FD6F8840021F000413D
:105820000143F9675FFA88F0BDE8F28F386840F409
:10583000801038607047002106F1200000F07DB82C
:105840000121301D00F006B80C10024090100240FB
:10585000007000402DE9F0410546794F28680C465C
:10586000F968002611F0030F0DD0F96801F003016B
:10587000814231D180B3F8686968C0F30210401CDE
:1058800088420ED028E0012804D025D303281DD05B
:1058900018D321E03A6891071ED5FA68696800F0CC
:1058A000C3F8386820F0806000F0C6F88046386899
:1058B000010113D502F07CF9A0EB08000328F6D310
:1058C000032637E039684A05E7D405E039688A03DA
:1058D000E3D439684A03E0D401262BE0A9682CB947
:1058E0003A695848EB6800F08FF80FE0012C3A69EC
:1058F00009D12B69544802405B0842EA01215B1E32
:1059000041EA435102E06B6900F084F8396138687C
:1059100040F0806000F090F804463868010105D43A
:1059200002F046F9001B0328F7D3C9E73869A969D3
:10593000084338613046BDE8F0812DE9F041064664
:105940003F4F30680C46F968002511F0030F0DD069
:10595000F96801F00301814231D180B3F8687168C0
:10596000C0F30210401C88420ED028E0012804D069
:1059700025D303281DD018D321E03A6891071ED5FE
:10598000FA68716800F050F8386820F0805000F034
:1059900053F880463868810013D502F009F9A0EB6E
:1059A00008000328F6D303252BE039684A05E7D41D
:1059B00005E039688A03E3D439684A03E0D4012555
:1059C0001FE0B1687A69002C04D11E48F36800F02A
:1059D0001BF802E0336900F01DF87961386840F087
:1059E000805000F029F804463868810005D402F0A0
:1059F000DFF8001B0328F7D3D5E7786971690843FE
:105A000078612846BDE8F081024042EA012141EA7E
:105A1000C36170470D4802405B0842EA01215B1EEA
:105A200041EA43617047000022F073021043491EAF
:105A300040EA0110F8607047386002F0B9B8000021
:105A400000100240FF80FF07FF809FFFFF80FFF9EB
:105A500070B508B9012070BD0268284D284CAA42D3
:105A600000F1240308D227498A181426B2FBF6F263
:105A700092001A62DC6108E023498A181425B2FBFF
:105A8000F5F2920021491A62D96102225A70016826
:105A90000D688168C26806686FF30E150D430169D1
:105AA000154342690D4381691543C2690D43016A7B
:105AB00015430D4335608268B2F5804F17D0DA691F
:105AC0000F21A2420CBF124A124A146893F82050C8
:105AD00005F01C05A94024EA01011160116893F842
:105AE0002040406804F01C04A040014311600020E5
:105AF000986101215970187070BD000008040240BF
:105B000000000240F8FFFDBFF8FBFDBF00040240AB
:105B1000A8000240A8040240F8B5044604F1240697
:105B200000253078012801D10220F2BD012030701B
:105B30007778012F26D1022070700027B761206886
:105B4000D0F800C04FEA5C074FEA470CC0F800C02D
:105B5000204600F0C4F82168F06820B10A6842F0DD
:105B60000E020A6008E0086820F00400086020685F
:105B7000016841F00A0101602068016841F00101FB
:105B8000016001E0357002252846F2BD00F12401D4
:105B90004A78022A05D00420886100220A70012078
:105BA00070470268136823F00E03136000680268F0
:105BB000520852000260012091F82020CB6902F0C7
:105BC0001C02904058600022012048700A7000209A
:105BD000704738B500F1240100244A78022A03D026
:105BE00004208861012417E00268136823F00E0383
:105BF0001360026815686D086D001560012291F848
:105C00002030CD6903F01C039A406A6001224A707B
:105C10000C70496901B18847204632BDF8B500F1E2
:105C200024010423CA6914680268156891F8206089
:105C300006F01C0603FA06F73C4210D06F070ED59B
:105C40001468A50603D4146824F00404146000F05A
:105C50003EF8C968002939D0BDE8F440084702235E
:105C600003FA06F73C4213D0AF0711D51468A50616
:105C700005D4146824F00A04146001224A7000F06C
:105C800026F800220A70896801B3BDE8F44008478D
:105C9000082303FA06F6344218D02B0716D51468E9
:105CA00024F00E041460012291F82030CC6903F036
:105CB0001C039A406260012301228A614B7000221A
:105CC0000A70096911B1BDE8F4400847F1BD91F8C7
:105CD0002020CC6902F01C0293406360704770B5CD
:105CE00090F84450066C012405F01C05AC4074602B
:105CF000046863608068102802D1A260E16070BD12
:105D0000A160E26070BD2DE9F04104000D46164629
:105D1000984608BF012034D004F17807786820B98C
:105D2000002139702046FDF7B1FB242078602068FF
:105D30000168490849000160606A10B1204600F01E
:105D400069FB204600F052FA01281AD020688168C9
:105D500041F4804181602068816821F400410D4355
:105D60008560206801686FF3194141EA465141EAB4
:105D70000841016000F007F82046BDE8F04100F05E
:105D8000ACBBBDE8F0812068016841F00101016011
:105D90007047000038B5040001D1012032BD04F184
:105DA0007805686808B900F017F800F01AF808B12B
:105DB00000F031F800F02CF8012804D000F004F8CD
:105DC00021F02A0116E032BD2068416821F490419B
:105DD0004160206881687047002129702046FDF7E6
:105DE00055BB2420686020680168490849000160AB
:105DF000606A7047816000F004F8BDE8324000F04E
:105E00006CBB2068016841F00101016020467047C9
:105E1000204600F0EBB9204600F0FCBA2DE9F8432B
:105E2000054605F150060C46F06A202817469946AB
:105E30003ED10CB1380001D101203AE0002070635E
:105E40002121F16201F0B4FE378080467780A86896
:105E5000B0F5805F04BF286900281ABF20460027DC
:105E60002746044611E00022802100F024F8D8B92A
:105E70002868002C12BF14F8011B37F8021BC1F36D
:105E8000080101857088411E718043467088CDF8F5
:105E900000900028E7D10022402100F00CF818B94A
:105EA0002020F062002004E02020F062032000E0C7
:105EB0000220BDE8F283284600F05CBB38B50346FB
:105EC000D3F8800020280AD109B1100001D10120A7
:105ED00032BD00F006F8BDE8384000F091BB02206A
:105EE00032BD00201866DFF800431868A0420CD0CD
:105EF0004068040209D5186850E8004F054644F090
:105F0000806445E800400028F5D1184670472868AD
:105F100000F1080151E8001F490800F10803490099
:105F200043E8001000287047F8B5054640F60F0C0E
:105F30002A68D369104613EA0C0F0668976805F1C2
:105F4000580406F0200003F020010BD1002918BFEF
:105F500000280ED02169002900F028812846BDE8DC
:105F6000F44008475FEAC77C04D4DFF8A4E416EAEB
:105F70000E0F78D05FEAC37C48BF5FEAC65E07D5E4
:105F80004FF0010CC2F820C0E26A42F00102E26266
:105F90009A070AD5FA0708D5D5F800E00222CEF80C
:105FA0002020E26A42F00402E2625A070AD5FA07A8
:105FB00008D5D5F800E00422CEF82020E26A42F0AD
:105FC0000202E2621A070BD508B9FA0708D5D5F81C
:105FD00000C00827CCF82070E26A42F00802E262B2
:105FE0001A0509D5730107D52E684FF40062326295
:105FF000E26A42F02002E262E26A002A32D000291C
:1060000018BF002803D0216909B128468847E06AF3
:1060100029688A68510602D410F0280F1DD028463E
:1060200000F048FB28688168480611D500F0C9F8DF
:10603000FCD1E06960B10FF2F5618163E069FFF7BF
:10604000C8FD00280ED0E069816BBDE8F440084728
:106050002846BDE8F24001F0BDBD284601F0BAFD7A
:106060000020E062F1BDA068012875D1D80673D583
:10607000F10671D51020106229688868410639D56B
:10608000E1690868406880B20028EBD0228890421D
:10609000E8DA6080086801688A0623D400F09FF877
:1060A00021F4807100F062FAF8D1FFF730FFFCD1E3
:1060B000286800F1080151E8001F00F1080321F0F1
:1060C000400100F07AF8F3D12020A0620021A16005
:1060D00000F085F821F0100100F048FAF8D1E069ED
:1060E000FFF754FD0220E06021886088091A89B218
:1060F00028462DE0218862886088891A00281CBF04
:1061000088B2002852D02A46106850E8003F054661
:1061100023F4907300F04BF8F6D100F000FB00F18F
:1061200008065B0046E800300028F6D12020A06277
:106130000023A3602361136853E8003F156823F030
:10614000100300F034F8F6D10220E06089B2104666
:10615000BDE8F44001F03FBDD80209D5790207D56A
:106160004FF4801010622846BDE8F24001F034BDC3
:10617000180607D5310605D56169B9B12846BDE8CD
:10618000F4400847580611D571060FD500F027F8DE
:1061900021F0400100F0EAF9F8D1202060620021EE
:1061A00061612846BDE8F24001F017BDF1BD45E848
:1061B00000300028704721F0800143E800100028DB
:1061C0007047296801F1080252E8001F286800F1B1
:1061D000080321F0400143E80010002870472868B8
:1061E00050E8001F0246704700800040F8B50446A2
:1061F000DFF8840622681368A168034020690B4316
:1062000061690343E0690B43034313600025516850
:10621000E06821F4405101435160A369DFF854164E
:106220008A421CBF206A03439668DFF85076DFF885
:10623000500626F4306633439360BA424FF400436D
:10624000DFF8406632D1366806F00306032E3BD8ED
:10625000DFE806F0027161840127E169B1F5004FC2
:106260004FF6F07640F0AB805FB1012F00F09F80D9
:10627000022F0AD0042F00F09D80082F00F09D808F
:10628000BFE0FEF759FA00280FD061684A0802EB18
:106290004002B2FBF1F0A0F11001B142F0D2064091
:1062A000C0F3420006432068C660ABE0DFF8D87553
:1062B000BA4221D1366816F00C0660D0042E3AD0CE
:1062C000082E28D00C2E49D010278A42C5D137B1CC
:1062D000022F08D0042F54D0082F55D091E0FEF79C
:1062E0002BFA0028E1D0626802EB4201884202D317
:1062F000130383424AD284E0DFF89075BA420CD18E
:10630000366816F030063AD0102E14D0202E02D067
:10631000302E23D0D8E70227D7E7DFF87475BA42CA
:106320000BD1366816F0C00629D0402E03D0802E3F
:10633000F1D0C02EEDE70427C7E7DFF85875BA4261
:106340000ED1366816F4407619D0B6F5807FF2D0BB
:10635000B6F5007FDFD0B6F5407FB5D10827B4E7AA
:106360008A42B1D1366816F4406608D0B6F5806F1F
:10637000E1D0B6F5006FCED0B6F5406FC9E7002783
:10638000A3E7FEF790F9ACE71846ACE7010E560814
:1063900016EB002069410023FBF792FBA0F540714A
:1063A000DFF8F42491422CD22168C8602AE0FEF77D
:1063B000CBF968E7FEF777F965E7184665E747B177
:1063C000012F16D0022F07D0042F15D0082F16D07A
:1063D00017E0FEF7B1F9A8B1616800EB5100B0FB1E
:1063E000F1F0A0F11001B1420BD2226880B2D0606E
:1063F00008E0FEF7A9F9EEE7FEF755F9EBE71846D6
:10640000EAE701250020A066E0662846F2BD00000C
:106410002001000490F824100A0706D5026853688A
:10642000416B23F400430B43536090F82410CA07D8
:1064300006D502685368816A23F400330B43536026
:1064400090F824108A0706D502685368C16A23F4BD
:1064500080330B43536090F824104A0706D5026836
:106460005368016B23F480230B43536090F824108E
:10647000CA0606D502689368816B23F480530B43E8
:10648000936090F824108A0606D502689368C16B61
:1064900023F400530B43936090F824104A0610D560
:1064A00002685368016C23F480130B435360036C40
:1064B000B3F5801F05D15368416C23F4C0030B432F
:1064C000536090F824100A0606D501684A68806C6B
:1064D00022F4002202434A607047F8B5054605F1F0
:1064E00078040020E0606FF07E4701F061FB064613
:1064F000286801680A0711D50097334600224FF437
:106500000011FFF7D8FC48B1FFF769FE21F08001C8
:1065100000F02CF8F8D12020606017E028680168AE
:106520004A0717D50097334600224FF48001FFF742
:10653000C2FC78B1FFF753FE21F4907100F016F819
:10654000F8D1FFF7E4FCFCD12020A06000212170ED
:106550000320F2BD202060602021A1600020286679
:10656000002169662070F2BD21F4F07142E800104C
:10657000002870472DE9F041069C05460E469046DE
:106580001F462868C1693140B1420CBF012000207C
:10659000404533D114F1010FF3D001F009FBC01BCA
:1065A000844200D314B90320BDE8F0812868016853
:1065B0004A07E6D5C169080704D42968C8690105F6
:1065C000DFD50DE02A6808201062284600F072F836
:1065D00005F178000821C160002202700120E3E784
:1065E00029684FF400600862284600F063F805F15E
:1065F00078002021C16000220270D4E70020D3E798
:1066000020B503460020596503F158010A804A80ED
:106610000861FF229868B0F5805F04D1186990B9CD
:1066200040F2FF120FE018B9186960B17F2007E04F
:10663000B0F1805F06D1186908B97F2203E03F20DE
:10664000888001E000228A800020C86222228A62BB
:10665000186800F1080252E8002F00F1080542F026
:10666000010245E800200028F2D19868B0F5805F6B
:1066700004BF186900280DD10FF215120A611868BD
:1066800050E8001F024641F02001FFF76FFFF6D1EE
:10669000002020BD0FF2A9020A6118690028EED07F
:1066A000196851E8001F1A6841F49071FFF75EFF06
:1066B000F6D1EDE710B500F00EF8FCD100F015F8BA
:1066C000FCD1016E00F01EF82021C0F880100022DD
:1066D0000266826610BD016851E8002F0B4622F465
:1066E000907243E8002100297047016801F1080217
:1066F00052E8002F520801F10804520044E800213A
:1067000000297047012909D1026852E8002F036867
:1067100022F0100243E800210029F5D170471068EB
:1067200000F1080353E8003F5B087047806A00F1FE
:10673000520100220A8100230B8001F04BBA0000B5
:1067400038B500F04DF81ED18B8C9188446D0B400C
:106750002370416D4B1C00F049F818D100F04DF842
:1067600000F060F8FCD100F06AF80BD100239360D0
:1067700000F04EF8FCD10168CB69DC0644BF102361
:106780000B628BE08FE0088B40F00800088331BD7E
:1067900038B500F025F81ED18B8C9188446D0B40E4
:1067A0002380416D8B1C00F021F818D100F025F8F2
:1067B00000F038F8FCD100F042F80BD100239360D0
:1067C00000F026F8FCD10168CB69DC0644BF102339
:1067D0000B6263E067E0088B40F00800088331BD7E
:1067E00000F158020168936A222B70474365518873
:1067F0004B1E5380518800297047036853E8003FBF
:10680000046823F4907344E800310029F5D17047FF
:10681000016851E8003F0C4623F0100344E80031C2
:1068200000297047016801F1080353E8003F5B0845
:1068300001F108055B0045E800310029704720217F
:106840009162002313610021D1600A4B01689942D3
:106850000CD049680B0209D5016851E8003F0C468D
:1068600023F0806344E800310029F5D191680129C3
:106870007047000000800040F369FFEF00380140DE
:106880000024F4008810024000440040004800400A
:10689000004C00400050004000FD0F001188BDE892
:1068A000344001F098B9BDE8324001F097B90000DA
:1068B00030B500F140025378202B0CD11478012C14
:1068C00009D000F01DF824F480541C6003681D6892
:1068D0002943196020E0022030BD30B500F14002AC
:1068E0005378202B0AD11478012C07D000F008F837
:1068F00024F4706444EA01241C600DE0022030BDE1
:10690000012313702424547003681D686D086D0002
:106910001D6003681C6870470068016841F0010150
:1069200001602020507000211170002030BD000057
:1069300038B5040001D1012032BD04F1400568786A
:1069400020B9002129702046FCF7F1FE00F044F840
:106950006068216820F0706008612068816821F417
:1069600000418160E0680128A0680CBF40F400404D
:1069700040F4044021688860E0680228206841688B
:106980000CBF41F4006121F400614160206841685E
:1069900041F0007141F4004141602068C16821F478
:1069A0000041C16060692169A2690143206841EA30
:1069B0000221C160206AE1692268014311602068F8
:1069C000016841F0010101600020686020216970C8
:1069D00020630021A97032BD2420687020680168FE
:1069E00049084900016070472DE9F84300F0B5F807
:1069F00059D12178012956D00120207001F0D8F812
:106A000000F0DEF800284CD1212000F0AFF8708DA6
:106A1000DFF81012B0F5807F03D335854FF0807317
:106A200004E0708D30854FF0007390B1706AD6F835
:106A300000C00278CCF82820706A421C7262708D07
:106A4000421E7285308D421E32850091521CD2B298
:106A500004E00091002201E000F0BCF800F0A4F88E
:106A600000F075F818D000F01BF9002819D100F0DB
:106A70008CF80028F4D089B20029F1D100F098F800
:106A800078B900F07EF8E7D2708D30850021009152
:106A90004FF00073328DDAE700F02FF900F0A1F823
:106AA00002D0012000E00220BDE8F2832DE9F84386
:106AB00000F053F843D12178012940D00120207003
:106AC00001F076F800F07CF8002836D1222000F0A2
:106AD0004DF8718DDFF85001B1F5807F28BF358505
:106AE00009D2718D318500904FF00073328DD2B292
:106AF00003E03585002000F025F800F055F800F09F
:106B000026F815D000F01AF9002816D100F07BF80D
:106B10000028F4D089B20029F1D100F049F860B919
:106B200000F02FF8E5D2708D308500210091DBE771
:106B300000F0E3F800F055F802D0012000E0022058
:106B4000BDE8F28300904FF08073FF227047708D94
:106B500000284A46394630467047064606F140044A
:106B600088466078202815461F46704760701021BF
:106B7000A17000206060756277857063FF25089FB3
:106B80007047708DB0F5807F7047706A3268017809
:106B90009162706A411C7162708D411E7185308DE9
:106BA000411E3185708D70474146304600F089B9ED
:106BB000CDF800903B4600228021304600F046B8D8
:106BC0008146CDF80090192301224FF40041304650
:106BD00000F03CB83585002000904FF08073FF2214
:106BE000704701000DD132682020D0613268DFF893
:106BF0003C00536803405360202262700020A07064
:106C00002070080070473068416A706A0170716ACC
:106C1000308D4A1C411E72623185708D421E728514
:106C2000708D7047002000800024008000E800FE86
:106C3000006881698A0744BF002181628169CA07AF
:106C400003D4816941F00101816170472DE9F04170
:106C5000069F05460E4690461C46286881693140CD
:106C6000B1420CBF01200020404517D114F1010FA3
:106C7000F3D000F09DFFC01B844201D3002CECD167
:106C8000286881693140B1420CBF01200020404595
:106C9000E3D100F026F80120BDE8F0810020FBE7F9
:106CA00070B505460C46164628688169880716D4D3
:106CB00000F040F818B914F1010FF5D001E00120FF
:106CC00070BD00F075FF801B844201D3002CEBD116
:106CD000286881698807E7D400F003F8EFE700200F
:106CE00070BD05F140002022416841F02001416063
:106CF0004270002181700170704770B505460C46E6
:106D0000164628688169880612D400F013F808B185
:106D1000012070BD00F04CFF801B844201D3002C89
:106D2000EFD1286881698806EBD4FFF7DAFFEFE737
:106D3000002070BD32462146284647E070B5054622
:106D40000C4616462868816948073DD4FFF7F2FFD4
:106D5000002837D12A68906981061ED590694107BD
:106D600001D5288D80BB9069C30605F1400104D58B
:106D70001020D06104224A6001E0002048602022F7
:106D80002868C2612A68584853680340536020222B
:106D90004A7000208870087014E000F009FF801B22
:106DA000844201D3002CCDD1286881694807C9D419
:106DB00005F140002022416841F02001416042700D
:106DC00000210170012070BD002070BD2DE9F84345
:106DD000044600252068836900269046DA0604F1FF
:106DE000400739D51023C36189462BE029002DD1F6
:106DF00019F1010F26D000F0DBFEA0EB0800814561
:106E000002D3B9F1000F1DD120684168BA788369B7
:106E10001B040AD5490408D4202A06D0416841F44D
:106E20008041416000F0C4FE804620688169880688
:106E300008D400F0BDFEA0EB08001A28F5D346F0F8
:106E400020060125206881698A06CFD50DB9202149
:106E5000C16146F00406012520688169CA0505D58F
:106E60004FF4807346F00106C3610125480506D53D
:106E700020684FF4806246F00806C261012588054B
:106E800007D520684FF4007146F00206C161012564
:106E900001E028000CD02046FFF7CAFE00F00BF8F6
:106EA000202079680E437E6078700021B9703970B7
:106EB0002846BDE8F28321680B484A6802404A60D0
:106EC000704770B50068049C4568084EC1F309011D
:106ED00041EA0241194346EA54562143B54321F0A1
:106EE00000412943416070BD00E800FEFF63FF03DD
:106EF00038B5040001D1012032BD606A30B9606844
:106F0000B0F5827F05D00021E16102E00020206120
:106F100060610020A06204F15C05687820B900215E
:106F200029702046FCF7B4FC0220687000F04AF893
:106F3000E168B1F5E06F04D90020B1F5706F03D1BD
:106F400004E04FF4805001D00021A1626168A26882
:106F5000237C01F4827102F404421143227D03F088
:106F600002031943A36902F001021143227F03F4D3
:106F70000073194394F8203002F038021143A26ADA
:106F800003F080031943236802F40052114319608F
:106F9000A16994F8242094F83430090C01F004011C
:106FA00002F010021143E26803F00803194302F4EF
:106FB0007062114308432168486000206860012125
:106FC000697032BD2068016821F04001016070479E
:106FD000016042600021C160002282600120704790
:106FE00010B5C2684368521C92FBF3F403FB1422F1
:106FF00083689A4202D16FF0010010BD0268C36835
:10700000D154C16800F014F8C160012010BD10B562
:107010008268C3689A4201D1002010BD026883686B
:10702000D45C0C70816800F003F88160012010BD11
:107030004268491C91FBF2F302FB131170470000F8
:1070400037B5044600250A460194009502AB01A914
:10705000074878441A30F9F7ACF8019A15700028FF
:107060004EBF04460198041B204603B030BD00BF4C
:107070007FA0FFFF38B5044600F09AFD14F1010F20
:10708000054602D004480178641800F091FD401BC9
:10709000A042FAD331BD00BFA8140020C0F3C751ED
:1070A00081B1FF2906D0C110400721F0E04101F174
:1070B0006051704741020CBF40F4E0016FF00041A5
:1070C0000020704700F0004100020AD0B0FA80FCB6
:1070D00000FA0CF001F16051A1EB0C5101EBD02151
:1070E00040057047F8B5D2B2022A3CD1C9B200249B
:1070F0004A1E18E000EB860500EB860795ED010AB5
:10710000D7ED000AB4EE600AF1EE10FA05D5CDED28
:10711000000A87ED000A009F6F60761C0D1B6D1E34
:10712000AE42E7DB641C9442B8BF0026F6DB0124C4
:1071300000930AE000EB83039DED000AD3ED000A03
:1071400070EE200ACDED000A641CE3B29342F1DB3D
:10715000891E00EE101AB8EEC00ADDED000AC0EE7E
:10716000800ACDED000A0098F2BD0000BFF34F8FFA
:10717000DFF84814DFF848040A6802F4E0620243CA
:107180000A60BFF34F8F00BFFDE730B503464FF6EF
:10719000FF70002400E0641CE2B28A4211D213F8AE
:1071A000012B5040082205046D0C00F0010001285D
:1071B000B2BF284685F4204080F00100521EF2D173
:1071C000E9E730BDDFF8FC03016802E0DFF8F40313
:1071D000416800EE101AF2EE040A20EE200ABDEE1D
:1071E000C00A10EE101A0804000E40EA012080B216
:1071F0007047DFF8D0038168EBE7DFF8C803C168A8
:10720000E7E7DFF8C0030169E3E7DFF8B8034169A6
:10721000DFE7DFF8B0038169DBE7DFF8A803C169C6
:10722000D7E7DFF8A003016AD3E74FF41060704797
:107230004FF42060704780B5FBF731FFDFF888031B
:107240004078000202BD80B5FBF729FFDFF8780324
:10725000418805E080B5FBF722FFDFF86C038188E9
:10726000080A40EA012080B202BD80B5FBF717FF93
:10727000DFF85403C188F3E7002070471FB5DFF83B
:107280004813008848700922684621E03EB500880E
:10729000DFF834436080684621460922F9F782FF0F
:1072A0006D4695E80700FBF7E9FE6088FCF7CEF82D
:1072B0006088FCF7B8F800203EBD1FB50088C249C1
:1072C000888003E01FB50088BF49C880684609224E
:1072D000F9F768FF6C4694E80700FBF7CFFE002043
:1072E00004B010BD80B50088012804D1012181F3CC
:1072F0001388FFF73BFF002002BD80B500880128FE
:1073000006D1FBF7E7FE012080F31388FFF72EFF7D
:10731000002002BDF8B50446AC4F15461E4632218A
:10732000384600F05DFCA84A507838700321797027
:10733000BE7032462946F81CF9F734FFB978C91CEB
:10734000C9B23846FFF721FFF91C88533946204659
:10735000BA78BDE8F840521DFCF724BB2DE9FC418A
:1073600005468878CE784C7946EA0026087944EAC2
:107370000024A6F109000B2801D3182E02DB3146A8
:107380009AA00AE03CB13019A0F10A010B2902D3FE
:10739000401E182804DB21469AA0FCF730FB3BE096
:1073A0009DA0DFF82C820088ADF80400FF21009139
:1073B000012301AAEE218748FFF716FBFCF758FDD1
:1073C000C8214046FBF7BAFC002707E0002002E096
:1073D00051680020884728F817007F1CA7420EDA62
:1073E000B919002082B208EBC202CBB252F8C8CF62
:1073F0006345EDD0401C82B2102AF3D3E6E776480D
:10740000016864008D4201D100F008F873480168FA
:107410008D4201D100F002F8BDE8F381A3B24246EB
:107420000321284676E700002DE9F8410F469BB07E
:107430000646B878FC787D7944EA00243879A4F1CE
:107440001401092945EA002502D3214667A006E078
:107450001DB160191538092804D3294669A0FCF725
:10746000CEFA41E0642102A8FBF768FC002009E0A5
:1074700007EB4001CA79097A41EA022102AA22F8FF
:107480001010401CA842F3DB4F48DFF854814178CC
:107490008DF80010042178788DF801008DF80240F5
:1074A0008DF803506846FFF770FE8DF80400062241
:1074B000000A8DF8050069463046FCF773FA00278C
:1074C00010E0002658F836003919884206D102AA81
:1074D00008EBC60102EB47004A689047761C062E6F
:1074E000F0D37F1CAF42ECDB1CB0BDE8F081F8B5F7
:1074F0000D461646044606F1FE01C9B22846FFF7BE
:1075000044FEA91911F8022D497842EA012290425D
:1075100014D16878032818BF10280FD10026314FE6
:10752000687857F83610884205D107EBC60229461D
:10753000536820469847761C022EF1D3F1BD2DE901
:10754000F0418046FCF73DFA50B31420FCF77EFD75
:10755000254C32212046FBF7F1FB312700261A4D3E
:107560004046FCF73BFAA055761C012E0BD1207843
:10757000697888421ED00022611C2046F9F712FE6D
:10758000761E7F1E16E0607803280BD1082E11D1DD
:10759000002E05DD324621464046BDE8F041A6E713
:1075A000BDE8F081102802BFA6F10900A179B0EB77
:1075B000410FEDD0BE42D3D3F2E700000CED00E066
:1075C0000400FA05D43D0020681400207C3A002015
:1075D000F0120020343B0020003400203035002021
:1075E00038140020E0120020083E002073746172FD
:1075F000745F7265675F61646472206572726F7236
:107600003A2564007265675F6E756D206572726FF2
:10761000723A256400000000FFFF0000F0B585B05D
:1076200050260B9D25B986F3118800F019FAFEE764
:107630000C9C24B986F3118800F012FAFEE7542757
:107640000097DDF800E0BEF1540F04D086F31188F6
:1076500000F006FAFEE7009E25630026022584F866
:10766000515004AF0A9D039602940197009500F0D3
:1076700034F8204600F06FF8049805B0F0BD2DE90D
:10768000F8430646174684B088469946B80000F08D
:10769000ABFA05001CD0542000F0A6FA040014D068
:1076A0000020256384F85100039002940D980C99F2
:1076B000019000914B463A464146304600F00DF8A5
:1076C000204600F048F8012004E0284600F014FBB2
:1076D0004FF0FF3005B0BDE8F0832DE9F0470A9E7A
:1076E0008046306B00EB8202101FC0084FEAC00AD0
:1076F00006F1340451B100228D5CA554885C10B1B0
:10770000521C102AF8D30020E07300E02170089F7B
:10771000062F88BF0627099DF76227610021616156
:107720009946301D00F045FB06F1180000F041FBC2
:107730003661C7F10707B76176620020A0610021BA
:1077400021774A464146504600F070FB306005B153
:107750002E60BDE8F0872DE9F04100F067F8DFF812
:10776000BC53DFF8BC83E86C401CE8641426A86AAC
:1077700028BBAC62E86C012829D1002706FB07F082
:10778000404400F009FB7F1C072FF7D305F174007C
:1077900000F002FB05F18807384600F0FDFA2846A4
:1077A00000F0FAFA05F1140000F0F6FA05F13800DD
:1077B00000F0F2FA05F17400E8622F6307E0A86DAB
:1077C00028B9E06AA96ACA6A904228BFAC62A86E6A
:1077D000401CA86600F096F94643211D08EB060000
:1077E00000F0EAFA00F0ADFBA86D30B100F03DF911
:1077F00003D200F09AF900F033F9BDE8F08180B5CA
:1078000088B1DFF81823116F21B100F03CF800F0C7
:1078100027F9FEE7116F491C1167002100F08BF971
:1078200000F03BF808B900F016F901BD044600F07D
:107830006FBB80B586B000210591049103AA04A90D
:1078400005A8FCF74DFB05980499029000220092D0
:1078500001910023039A0FF250310FF21920FFF724
:10786000DDFE70B100F00FF800F0FAF8DFF8280341
:107870004FF0FF31C166012282650021016500F0F1
:10788000F7FA07B000BD502080F311887047DFF889
:107890000803016F491C0167704770B5DFF87C620F
:1078A000306F0024002520B900F044F800F0D8F82B
:1078B000FEE700F02DFB306F401E3067306F002870
:1078C00037D1F06CD8B934E0F068C46800F036F80D
:1078D00000F015F9E06A716DDFF8B83201228240DC
:1078E0001143716514225043211D184400F064FABD
:1078F000E06AB16ACA6A904224BF012131663068E9
:107900000028E1D10CB100F0EDF8F46D44B100F0C5
:1079100019F808B101203066641EF8D10020F06526
:10792000306E30B1DFF874124FF08050012500F056
:1079300096F8EEE0502181F31188704704F11800A9
:1079400000F060BA2DE9F843DFF8D071386F0026F7
:10795000002853D13C6D641C3C6510D1F86A006866
:1079600020B1FFF7E7FF00F07BF8FEE7F86A396B1C
:10797000F9623863786E401C786600F0B3F8F86EF0
:10798000DFF8109284424FF0140828D320E0F96AFF
:10799000C868C568686884422ED3281D00F032FA92
:1079A000A86A18B105F1180000F02CFAE86A796DA0
:1079B000012282401143796508FB00F0291D4844EB
:1079C00000F0FAF9E86AB96ACA6A904228BF01264B
:1079D000F86A00680028DAD14FF0FF31F966B86A1A
:1079E000C06A08FB00F859F80810022928BF0126D0
:1079F000386E30B1012604E0F866F0E7F86D401CFF
:107A0000F8658FE0DFF81421106F10B101211166C5
:107A1000704710661421506DB0FA80F3C3F11F0354
:107A20004B43DFF87011C85838B9502181F31188E1
:107A3000BFF34F8FBFF36F8FFEE7C81800F1080345
:107A4000416849684160994204BF496841604068A3
:107A5000C16891627047DFF844114FF080500860B0
:107A6000BFF34F8FBFF36F8F7047A86AC16AE06A98
:107A70008142704770B5DFF8A840DFF81C5111E073
:107A800000F046FA286AC668301D00F0BBF9E86CC1
:107A9000401EE864686B401E686300F052FA30468E
:107AA00000F009F8686B0028EAD121680229F9D3AF
:107AB000FFF7D1FFF6E710B5044694F8510040B93E
:107AC000206B00F019F92046BDE8104000F014B911
:107AD00010BD0128F7D00228FAD0FFF7D4FEFFF737
:107AE000BFFFFEE70D49C86A006810B94FF0FF32CA
:107AF00003E0C86AC268D0684268CA667047201D41
:107B000000F080B90122E06A696D82401143696525
:107B1000704700F016FA284670BD0000603600205D
:107B2000FC3600203046BDE8F2831C4A4FF08051FD
:107B3000116070470000F8B5174D2F6D0C46A96A0B
:107B40000646081D00F05EF930B9A86A696DC06A82
:107B5000012282409143696516F1010F05D124B1DC
:107B6000A86A011D05F138001AE0A86AF6194660F6
:107B7000BE42A86A05D2011D286BBDE8F44000F0A2
:107B800028B9011DE86A00F024F9E86E864238BF82
:107B9000EE66F1BDFC3600206036002004ED00E00A
:107BA000BDE8F44000F008B949444C45000000002D
:107BB00001484068704700BFA81400204018491CC5
:107BC0001CBFB1F1010100F8012DF9D170477047D8
:107BD00070477047704770477047704770470000A4
:107BE0000022FFF7EBBF00002DE9F8430446FFF742
:107BF0004EFE684FB8684FF00009002500BB07F142
:107C0000200307F1200113F0070F40F6B8300A46B1
:107C100004D0CA1DD208D200831AC81880180838A8
:107C2000C008C0003A607D60B86045600560831A96
:107C30005360106050683861F8604FF00040F861A0
:107C40004FF05008F869044246D1002C44D0083463
:107C500014F0070F04D004F1080104F007000C1A17
:107C6000002C39D0F868A04236D33E68394601E08E
:107C7000314606467068A04202D230680028F7D12B
:107C8000B868864228D00A683068086002F108099E
:107C90007268121B112A0CD3311911F0070002D09F
:107CA00000F023F8FEE7301D02517460084600F032
:107CB0004DF87168F8683C69401AF860FA68A242A9
:107CC00088BF2246F8693A6101437160356009F066
:107CD00007057869401C7861FFF7DFFD15B100F0FA
:107CE00004F8FEE74846BDE8F28388F31188BFF345
:107CF0004F8FBFF36F8F7047002800D1704738B5A2
:107D0000A0F10805234C6968E2695023114204D1AF
:107D100083F31188FFF7EBFFFEE7286820B183F3B8
:107D20001188FFF7E4FFFEE791436960FFF7AFFDBD
:107D3000E16868684118E160284600F007F8A0692A
:107D4000401CA061BDE83140FFF7A7BD30B5114927
:107D50000A4600E01A4613688342FBD35368D418DE
:107D6000844203D14068C3185360104643681468C6
:107D7000C518A54208D189688C4204D06168CB1827
:107D80004360246800E00C460460824218BF106023
:107D900030BD0000D42500204FF0FF3200F1080173
:107DA00082604160C16000F108020261002101604F
:107DB000704700210161704710B542684A609368BE
:107DC0008B6094686160916008610168491C016082
:107DD00010BD30B50A6812F1010F08BF036907D062
:107DE00000F1080300E023465C682568AA42FAD245
:107DF0005A684A6091608B60596008610168491C4B
:107E0000016030BD4368016982689A608368426896
:107E10005A604A68824204BF83684B600022026154
:107E20000868401E0860086870470000490810B5DF
:107E30004900A0F120034FF0807499611A60DC6161
:107E40006FF002020FF20D01596140F8242D203825
:107E500010BD00004D494A68502012F1010F80F317
:107E60001188BFF34F8FBFF36F8F00D0FEE7FEE79F
:107E70007CB5474A474B10685021984202D100F028
:107E800093F8FEE71068444B984202D100F08CF85A
:107E9000FEE7424B1C780194FF251D701E783B4C79
:107EA0008DF800609DF8000000F050002070072061
:107EB00005E09DF800506D00401E8DF800509DF8C3
:107EC00000502E06F5D4454215F1030F03D0A060F3
:107ED00000F06AF8FEE7000200F4E060A06001989C
:107EE0001870116A41F470011162106A40F070401C
:107EF000106200F061F80020606000F0BBF82848D4
:107F0000016841F04041016000F0A4F8002076BD16
:107F1000502080F31188BFF34F8FBFF36F8F1B4941
:107F20004A68521C012A4A600AD11E490A6813068F
:107F300006D080F31188BFF34F8FBFF36F8FFEE73A
:107F400070471249486838B9502080F31188BFF350
:107F50004F8FBFF36F8FFEE7401E486008BF80F36E
:107F60001188704780B5502080F31188BFF34F8F80
:107F7000BFF36F8FFFF7E6FC18B10A494FF080504E
:107F80000860002282F3118801BD000074140020F3
:107F900000ED00E071C20F4170C20F4100E400E04B
:107FA00034EF00E004ED00E081F31188BFF34F8F60
:107FB000BFF36F8F704700000748084B0021016036
:107FC0000022826028221968B1FBF2F2521E426040
:107FD00007210160704700BF10E000E0D4140020CA
:107FE000EFF30980BFF36F8F264B1A681EF0100F56
:107FF00008BF20ED108A20E9F04F106009B44FF05F
:10800000500080F31188BFF34F8FBFF36F8FFFF7DE
:10801000F9FC4FF0000080F3118809BC196808686A
:10802000B0E8F04F1EF0100F08BFB0EC108A80F3DC
:108030000988BFF36F8F7047124B19680868B0E862
:10804000F04F80F30988BFF36F8F4FF0000080F38B
:10805000118870470C480068006880F308884FF06A
:10806000000080F3148862B661B6BFF34F8FBFF390
:108070006F8F00DFDFF81400016841F470010160C8
:10808000704700008836002008ED00E088ED00E031
:1080900080B52DED068BB0EE409AF0EE418AF6EEFB
:1080A000009A39EE280AB0EE608A20EE290A80EEA6
:1080B000080A00F0CFFBB0EE40AA00F0E3FC79EE36
:1080C000680A60EEA90AC0EE880A80EE800A00F015
:1080D000DBFC80EE0A0ABDEC068BB1EE400A01BD66
:1080E0002DE9F0412DED028B82B0804601AB6A464E
:1080F00000F0EEFCDFF800770198BDF80010786121
:1081000039802D23BDF90000C0EB0012642110FB63
:1081100003F3002592FBF1FE502210FB02F093FBCB
:10812000F1F6019B90FBF1FC1FFA8EFEB6B21FFA2E
:108130008CFC462B28BFA3F146052B46012204E008
:10814000B442A8BFA44543DA5B1C019883425CD2C9
:1081500008EB4300011FB1F90240B1F90050A542FC
:10816000F2DAB0F90050A542A4BFB0F90240A5422E
:10817000EADBB0F90450A542E6DA07F1140444F84A
:108180002230058827F81250521CB0F9004074457F
:10819000A8BFA642D4DBB0F90200B1F9021000EE8C
:1081A000103A00EE900AB8EE408AB8EEE01A00EEFF
:1081B000904A00EE101AF8EEE00AB8EEC00AFFF797
:1081C00067FF38EE000A02B0BDEC028BBDE8F0811B
:1081D00000EE103AB0F90200B1F90210B8EE408A90
:1081E00000EE100AB8EEC01A00EE104AF8EEC00A0F
:1081F00001EE901AB8EEE10AFFF74AFF38EE000AE6
:10820000FAEE090A30EE200ADDE79FED820ADAE78E
:1082100038B50446DFF8205600224FF4E07100F034
:108220002AF800224FF4604100F025F8641E032C68
:1082300020D8DFE804F002060F1701224FF40051A6
:1082400013E001224FF4807100F015F801224FF481
:1082500080410AE00122802100F00DF801224FF454
:10826000C04102E001224FF4C0712846BDE8384009
:10827000FAF74EBE31BD2846FAF74ABEF8B50546B4
:108280000E46FAF7DEFADFF87445DFF8747520461B
:10829000F9F7EAFC21680020486232462946DFF8F7
:1082A0006405FCF7EDFD3868016A41F2111640F2F1
:1082B0004445314204BF016A294200F024F80021FC
:1082C0004162012080F31088DFF87005F9F740FD66
:1082D0003868016841F001010160416AB1F5827FAF
:1082E000FBD3016A314204BF016A294200F00BF856
:1082F0002046F9F784FC002080F31088BDE8F240A6
:108300000120FBF7A3BE03D10268520852000260AD
:10831000704700002DE9F8432DED028B82B0054631
:108320000C4616460C9F98460DF10202322130464B
:1083300000F00AFC6A463221404600F005FCBDF917
:108340000210DFF8C49449423B46324609B2304637
:1083500000F022FCBDF9001049423B46424609B2FA
:10836000404600F019FC39463046FFF7B9FEF0EE02
:10837000040ADFED298A80EE200AB9EE048A30EE85
:10838000280A30EE080A89ED000A39464046FFF710
:10839000A7FEB0EE041A80EE011A31EE281A31EE73
:1083A000080AD9ED000A89ED010A70EEC01AC9ED7C
:1083B000021AB7EE001AF7EE001AC1EE200A81EE9B
:1083C000800A30EE800A9FED152A20EE022A12EE76
:1083D000100A9FED971AE860DFED111AD9ED020A35
:1083E00099ED000A20EE811AC1EE211AC1EE801A21
:1083F00081EE800A2CB9B1EE400A10EE100A286016
:1084000002E010EE100A686002B0BDEC028BBDE81D
:10841000F1830000000000000000824300606A4712
:108420002905B53F2DE9F84F2DED068B84B0DFF817
:10843000DCA30AF6CC010AF1CC0201240AF1C00740
:10844000029101929FED7B9ADFF8C463DFF8C45379
:1084500041F2111B2868016A11EA0B0F02BF016A81
:1084600040F24442114200F0F7F8002242620168F3
:1084700041F0010101600120FFF7CAFE00F0F2F8AF
:108480000120FBF7E3FD0220FFF7C2FE00F0DAF85F
:1084900000F0D2F800215046FFF73CFF0320FFF721
:1084A000B7FE00F0DFF80120FBF7D0FD0420FFF756
:1084B000AFFE00F0C7F800F0BFF801215046FFF70B
:1084C00029FFDAED008A9AED018A28EEA80A08EE63
:1084D000080A00F08BFB8AED020A18EE900ADAED2A
:1084E000029AFEF7DBFD8046894619EE900AFEF7F8
:1084F000D5FDDFF82423DFF82433F8F797FF00F0E9
:10850000A5F800F083FB00EE100A00F0A3F98AED55
:10851000040A2868016A11EA0B0F02BF016A40F2DF
:108520004442114200F098F8DFED5F0A38680AEB28
:108530008001C1ED1C8A81ED268AC1ED089A9FED6C
:108540005B1A9AED040A60EE200A80EE811A81ED32
:10855000121A401C0A28386055D3002038600AF1EE
:10856000C4020A210AF1700000F084FB0AF1C8027B
:108570000A210AF1980000F07DFB97ED01AAD7EDE2
:1085800002AA2AEE0A0A0AEEAA0A00F02FFBF0EE6F
:10859000409A19EE900AFEF781FD41EC180B1AEE95
:1085A000100AFEF77BFD8046894653EC182BDFF856
:1085B0007002DFF87012F8F739FF00F047F800F0AA
:1085C00025FB00EE100A00F045F9DFED390A80EED8
:1085D000200AF5EE40AA20EE09AAF1EE10FA48BFF3
:1085E00039EE4AAA51EC180B21F000418E4A8F4B0C
:1085F000F8F71CFE3CBFDFED7F9A9FED7EAAC6ED2B
:108600000B9A86ED0CAA2620FBF720FD002C0ED03D
:1086100000249AED030A86ED000A86ED010AB46093
:108620009AED020A86ED030A86ED040A746111E7E9
:108630000060EA470000B4434FF480600090029B62
:10864000019A704702984FF4806117E602460B4684
:1086500040464946F9F71AB803D10168490849006C
:108660000160704701984FF4806107E670B52DED09
:10867000028B05460C469FED728B00260AE055F8EA
:108680002600FEF70BFD53EC182BF8F7CFFE41EC5C
:10869000180B761CA642F2DBB0EE480AF0EE680A30
:1086A000BDEC028B70BD000000003443DB0F49407D
:1086B000DB0FC94070B55F4800F596552DED048B72
:1086C000296800EB810200F5166682ED000A4FF47E
:1086D00016722B6806EB83011446C1ED000A2B6865
:1086E00069685B1C93FBF4F402FB14332B60B1F557
:1086F000167FB8BF491CB1F5167FC8BF1146696027
:10870000FFF7B4FF6C68B0EE408AF0EE608A204656
:10871000F8F77AFE02460B4651EC180BF8F7B6FF55
:1087200000F074FA08EE100A85ED028A2146304600
:10873000FFF79CFF6868B0EE409AF0EE609AF8F799
:1087400063FE02460B4651EC190BF8F79FFF00F051
:108750005DFAD5ED060AF4EE480A00EE100AF1EED5
:1087600010FA48BF85ED068AD5ED070AF4EE400AF7
:10877000F1EE10FA48BF85ED070AD5ED040AB4EE14
:10878000608AF1EE10FA48BF85ED048AD5ED050A3E
:10879000B4EE600AF1EE10FA48BF85ED050A1C48F8
:1087A0006969016080ED010AE96981602A69C26036
:1087B00080ED048AA969416185ED030ABDEC048B53
:1087C00070BD70B5124D00F03FF80024184E4FF404
:1087D0007A70FBF73BFCF088641C844202DB00F0FB
:1087E00033F80024D5ED0C0A95ED0B0AFFF762FF74
:1087F000EDE7000000000000983D0020203C002034
:108800006C3C0020B03900204C3E002008150020B0
:10881000D43D0020043D00202D431CEBE2361A3FDE
:108820003A8C30E28E79453E9A9999999999B93F57
:10883000681400200000002000080048B83C002018
:10884000000000000000000005F11C0105F1180007
:10885000FBF768BA10EE101A04204FF07E5201EEBA
:10886000902A490088BF0820490800EE101A91425A
:1088700014D871EEC00A0F4A31EE801A914261EEAF
:10888000200AF1EEE00A05D980F0040080EE800AAB
:1088900000F0ACBA80EE200A00F0A8BA490011F14D
:1088A000807F9CBF6FF0004100EE101AAFF3008094
:1088B00070470000F404353FDFED620A60EE200AE5
:1088C00010EE902A22F0004101EE101ADFED5E1A40
:1088D000B4EE611AF1EE10FA25D54FF07C5102F09A
:1088E00000420A4301EE102A71EE200AFDEEE00A72
:1088F00010EE901A00296AD0FAEEC90A9FED531AB9
:1089000000EE810ADFED521A00EEA10A9FED512A16
:1089100000EE820ADFED502A00EEA20A9FED4F1A08
:1089200000EE810A53E010EE101A4B001B1613F1F3
:10893000010F0AD14900081610F1010F02D10902F6
:1089400040F07F809FED460A7047490004D100281F
:1089500077D0B7EE000A70474FF07C5102F000422A
:108960000A4301EE102A71EE200A10EE902A5100FF
:108970000DD0090EC1F196011829A8BF02F00042DE
:1089800003DA0029C4BFCA408A4000EE902A10EEE4
:10899000901A490017D09FED331A20EE811ADFEDAF
:1089A0002B1A01EE210A9FED2A2A01EE020ADFEDC1
:1089B000292A01EE220A9FED283A01EE030ADFED93
:1089C000271A01EE210AFDEEE00A10EE901A01F0DE
:1089D0000301081810EE101A21F0004100EE901A61
:1089E0009FED211AF4EE410AF1EE10FA04D5C10709
:1089F00023D5B7EE000A20E0C10760EE000A0ED5CD
:108A00009FED1A0A9FED1A1A00EE801ADFED191A6F
:108A100041EE201AB7EE000A01EEA00A0DE09FED2C
:108A2000162ADFED161A40EE821ADFED152A20EE27
:108A3000201A41EEA02A01EE220A800748BFB1EEBB
:108A4000400A704783F9223F0000004F0000C9C66A
:108A500000A0FDC00020A2BA000034B30030C2AEB6
:108A6000FFFFFF7F00008038000080399349B2BAD1
:108A700036A02A3DDFFFFFBE6E8C4CB94283083C16
:108A8000A1AA2ABE002017E710EE101AC1F3C752A0
:108A9000DAB1992A0FDAC80F21F0004100EE101A5E
:108AA000B1F17E5F40F3A281F7EE000A80EE800A0A
:108AB000001D00F09BB9FF2A01D14A0205D1034AEB
:108AC000C90F42EAC17100EE101A7047DB0FC93FAF
:108AD000F0B50D4604466F1E002034F9026BB9084C
:108AE00084461FD0B4F900E07645BCBF76460CF151
:108AF0000100B4F902E07645BCBF76460CF10200F5
:108B0000B4F904E07645BCBF76460CF10300B4F935
:108B100006E008340CF1040C7645BCBF764660468E
:108B2000491EDFD117F0030C0BD0614634F9027BEC
:108B3000BE42BCBF3E46A5EB0C00491EACF1010C89
:108B4000F4D116801860F0BD70B403460024880884
:108B500081B012D01E68009635462E0404EB2644E0
:108B60005E68009604EB2544354608332E0404EB7A
:108B70002644401E04EB2544ECD111F0030004D040
:108B800033F9025B6419401EFAD194FBF1F01080B6
:108B900001B070BC70470000F0B40446980881B082
:108BA000C1EA014511D0276800973E4696FA15F6AE
:108BB00000961660676800973E4696FA15F600968E
:108BC000566008340832401EEDD113F0030F09D06F
:108BD00003F0030334F9020B90FA11F05B1E22F844
:108BE000020BF7D101B0F0BC70470000B5EEC00A2F
:108BF000F1EE10FA02D4B1EEC00A70476FF0004CEB
:108C000000EE10CAAFF300807047000001F0004290
:108C10008B1AA3F16051B1F5801F0ADBB1F17F6FB0
:108C20001FD242EAC102C10071F1004142EB507013
:108C300070470B15C3F10903212B10D2890241EAB9
:108C4000905180020128494141F0004121FA03F08E
:108C5000C3F12003994071F1004150417047100069
:108C600070476FF0000013EB103F5CBF000E42EA4C
:108C7000C05070478446880881B09FED5B0A00F0C1
:108C80009E8010F0030313D0DCED000A9CED011A66
:108C900030EE200A30EE010ADCED020A9CED031AE8
:108CA00030EE200A5B1E30EE010A0CF1100CEBD105
:108CB0005FEA900000F08380DCF800300093401EF3
:108CC000DCF80430DDED000A009330EE200ADCF819
:108CD0000830DDED000A009330EE200ADCF80C309D
:108CE000DDED000A009330EE200A0CF11003DDEDFB
:108CF000000AD3F800C0CDF800C030EE200AD3F847
:108D000004C0DDED000ACDF800C030EE200AD3F833
:108D100008C0DDED000ACDF800C030EE200AD3F81F
:108D20000CC0DDED000ACDF800C030EE200A53F88B
:108D300010CFDDED000ACDF800C030EE200AD3F8E8
:108D400004C0DDED000ACDF800C030EE200AD3F8F3
:108D500008C0DDED000ACDF800C030EE200AD3F8DF
:108D60000CC0DDED000ACDF800C030EE200A53F84B
:108D700010CFDDED000ACDF800C030EE200AD3F8A8
:108D800004C0DDED000ACDF800C030EE200AD3F8B3
:108D900008C0DDED000ACDF800C030EE200AD3F89F
:108DA0000CC0DDED000ACDF800C030EE200ADDED8C
:108DB000000A30EE200A03F1100C7FF47DAF11F0B1
:108DC000030007D0DCED000A401E30EE200A0CF153
:108DD000040CF7D100EE901AF8EE600A80EE200A3B
:108DE00082ED000A01B07047000000001AA210EEE8
:108DF000101A43F2A40CC3F6896CF2EC060A614522
:108E000009DB00EE803A70EE800A83EE200A40F023
:108E1000020010EE101A4900D1F1E6410BD860EEC5
:108E2000000A20EE203A03EE010A01EEA02A42EEEB
:108E3000202A80EE220A400810F0020F18BFB1EE7F
:108E4000400A02EB8002D2ED000A30EE200A28BF71
:108E5000B1EE400A70470000D7B3DD3F6AD5033F4B
:108E60002B94A93DB82A593F0000803F000080BFE5
:108E700000000000920A063FDB0FC93F920A863FBE
:108E8000DB0FC93F920A0640DB0F4940368D274071
:108E900000000000000000000000000000000000D2
:108EA00000000000000000000000000000000000C2
:108EB00000000000000000000000000000000000B2
:108EC00000000000000000000000000000000000A2
:108ED0000000000000000000000000000000000092
:108EE0000000000000000000000000000000000082
:108EF0000000000000000000000000000000000072
:108F00000000000000000000000000000000000061
:108F10000000000000000000000000000000000051
:108F20000000000000000000000000000000000041
:108F30000000000000000000000000000000000031
:108F40000000000000000000000000000000000021
:108F50000000000000000000000000000000000011
:108F60000000000000000000000000000000000001
:108F700000000000000000000000000000000000F1
:108F80005B4552524F525D205B25733A25645D204C
:108F9000417373657274696F6E2028726574203D29
:108FA0003D2048414C5F4F4B29206661696C6564E8
:108FB00021207368743330B2C9D1F9CAA7B0DC0A72
:108FC0000D0A00005B4552524F525D205B25733AFB
:108FD00025645D20417373657274696F6E20282863
:108FE000746D705F74656D646174612E6656616C3A
:108FF0007565203E3D202D343029202626202874FA
:109000006D705F74656D646174612E6656616C7518
:1090100065203C3D2038352929206661696C6564EE
:1090200021207368743330CEC2B6C8D6B5D0A3D170
:10903000E9CAA7B0DC0A0D0A000000005B455252E5
:109040004F525D205B25733A25645D204173736543
:109050007274696F6E202828746D705F68756D6911
:10906000646174612E6656616C7565203E3D2030EA
:10907000292026262028746D705F68756D696461EB
:1090800074612E6656616C7565203C3D2031303030
:109090002929206661696C65642120736874333006
:1090A000CAAAB6C8D6B5D0A3D1E9CAA7B0DC0A0D02
:1090B0000A000000FEE7FEE7FEE7FEE7FEE7704776
:1090C0002548FCF7ABBD80B52448F8F709FFBDE89B
:1090D00002402348F8F704BF38B5224D224C2846F9
:1090E000FCF722FF012221462846FCF7E7FE1F4835
:1090F00000684169C268491C91FBF2F302FB13113D
:109100000269914205D02178BDE834400830FDF76E
:1091100067BF31BD70B5164E164D3046FCF704FFE3
:1091200015490C68012229463046FCF7C7FE6069E4
:10913000E168401C90FBF1F201FB120021698842BA
:1091400006D0297804F10800BDE87040FDF748BF5B
:1091500070BD0A48FCF7E8BE503D0020883B002067
:10916000043D002088370020103800200034002003
:10917000143800209C38002030350020A038002012
:10918000453A5C595C4941525C6D6963726F5F633B
:109190006C696D6174655C447269766572735C5369
:1091A000687433785C73687433302E630000000099
:1091B0005B4552524F525D205B25733A25645D201A
:1091C000417373657274696F6E20286765745F748C
:1091D000656D705F68756D695F6461746128267480
:1091E000656D702C202668756D6929292066616976
:1091F0006C6564212021212153656E736F722053A9
:109200006874333020436865636B204661696C6520
:10921000640A0D0A0000000053656E736F722053DC
:109220006874333020436865636B204F4B2E0D0A02
:109230002054656D703A252E32662C48756D693A5A
:10924000252E32660D0A00000E48016841F47001B7
:10925000016000220C49086840F0010008608A6043
:109260004FF480520B68094803400B60CA6000202D
:109270000B68074A23F480230B6088614FF000617C
:109280001160704788ED00E000100240FFFFF6EA31
:1092900008ED00E0000000000000000001020304EF
:1092A00006070809453A5C595C4941525C6D69639F
:1092B000726F5F636C696D6174655C4170705C5363
:1092C00072635C696E666C6173682E6300000000F7
:1092D0005B4552524F525D205B25733A25645D20F9
:1092E000696E666C61736820657261736520657272
:1092F000726F72210D0A000030B4002512E050F8A0
:10930000042BD30744BF4A44521E091F042942F8C4
:10931000045BFAD213468C0744BF15809B1CC90717
:1093200048BF1D7050F8041B0029E8D130BC7047BD
:10933000A0860100400D0300801A060000350C00D5
:1093400040420F0080841E0000093D0000127A0098
:109350000024F40000366E010048E801006CDC02D5
:1093600010B5074979441831064C7C44163404E0A2
:109370000A68081D114488470146A142F8D110BD72
:109380002C000000480000004EF68851CEF200018B
:10939000086840F470000860BFF34F8FBFF36F8F11
:1093A0004FF00170E1EE100A704700004DFFFFFF23
:1093B0005C29000008150020000000009F7CFFFFD2
:1093C000FC010000F80100000000002000F00DF892
:1093D000002801D0FFF7C4FFAFF300800020AFF3F7
:1093E0000080F9F763FB00F002F80120704700F0FD
:1093F00001B8000007463846F8F7EAFBFBE7000033
:109400000548014603B4684680F30988AFF300803D
:10941000FFF7BAFFFFF7DAFFA5EDF5FE74656D689B
:10942000756D5F7570646174655F7461736B000066
:10943000014880470148004749920008019400080C
:1094400064656661756C745461736B00616E656D03
:109450006F6D6574657200006C65645461736B00B8
:109460000000000001020304FFF7FEBFFFF7FEBF8C
:10947000FFF7FEBFFFF7FEBFFFF7FEBFFFF7FEBF20
:10948000FFF7FEBFFFF7FEBFFFF7FEBFFFF7FEBF10
:10949000FFF7FEBFFFF7FEBFFFF7FEBFFFF7FEBF00
:1094A000FFF7FEBFFFF7FEBFFFF7FEBFFFF7FEBFF0
:1094B000FFF7FEBFFFF7FEBFFFF7FEBFFFF7FEBFE0
:1094C000FFF7FEBFFFF7FEBFFFF7FEBFFFF7FEBFD0
:1094D000FFF7FEBFFFF7FEBFFFF7FEBFFFF7FEBFC0
:1094E000FFF7FEBFFFF7FEBFFFF7FEBFFFF7FEBFB0
:1094F000FFF7FEBFFFF7FEBFFFF7FEBFFFF7FEBFA0
:10950000FFF7FEBFFFF7FEBFFFF7FEBFFFF7FEBF8F
:10951000FFF7FEBFFFF7FEBFFFF7FEBFFFF7FEBF7F
:10952000FFF7FEBFFFF7FEBFFFF7FEBFFFF7FEBF6F
:10953000FFF7FEBFFFF7FEBFFFF7FEBFFFF7FEBF5F
:10954000FFF7FEBFFFF7FEBFFFF7FEBFFFF7FEBF4F
:10955000FFF7FEBFFFF7FEBFFFF7FEBFFFF7FEBF3F
:10956000FFF7FEBFFFF7FEBFFFF7FEBFFFF7FEBF2F
:10957000FFF7FEBFFFF7FEBFFFF7FEBFFFF7FEBF1F
:10958000FFF7FEBFFFF7FEBFFFF7FEBFFFF7FEBF0F
:10959000FFF7FEBFFFF7FEBFFFF7FEBFFFF7FEBFFF
:1095A000FFF7FEBFFFF7FEBFFFF7FEBFFFF7FEBFEF
:1095B000FFF7FEBFFFF7FEBFFFF7FEBFF2FF0001A0
:1095C000F1FF01F1FF01F1FF01F1FF01F1FF01F1F5
:1095D000FF01F1FF01F1FF01F1FF01F1FF01F1FFD7
:1095E00001F1FF01F1FF01F1FF01F1FF01F1FF01C5
:1095F000F1B00143C84304410112030910035D7334
:1096000000081008FC02BB29740008F0121003C502
:1096100071000801D112CD0812020812F30821F0DE
:1096200012FB081204081003037200080508120B4D
:1096300008120608121308120708121B082509123F
:109640002308120908122B08120A081231081214F2
:109650000812370812150812470812160812550882
:10966000121708126B08121808527928527D2852D6
:109670008D2852BB2812C508121A0812E508121BC1
:109680000812FB0840085530802558025802160081
:109690000112AA01F212000150078800062C062CC4
:1096A0000000012DF2021035E2011433093D15F3DB
:0896B0000280252DF2050318CC
:04000005080094015A
:00000001FF
